:020000040100F9
:1000000038480020E5000001ED000001EF0000018C
:1000100000000000000000000000000000000000E0
:10002000000000000000000000000000F1000001DE
:100030000000000000000000F3000001F5000001D6
:10004000F7000001F7000001F7000001F7000001D0
:10005000F7000001F7000001F7000001F7000001C0
:10006000F7000001F7000001F7000001F7000001B0
:10007000F7000001F7000001F7000001F7000001A0
:10008000F7000001F7000001F7000001F700000190
:10009000F7000001F7000001F7000001F700000180
:1000A000F7000001F7000001F7000001F700000170
:1000B000F7000001F7000001F7000001F700000160
:1000C0000348854600F056F80048004751050001F6
:1000D0003848002040BA7047C0BA70470138FDD197
:1000E000704700000448804704480047FEE7FEE7E9
:1000F000FEE7FEE7FEE7FEE795030001C100000111
:1001000030B50B46014600202022012409E00D46AF
:10011000D5409D4205D31D469540491B2546954037
:1001200040191546521E002DF1DC30BD03460B432D
:100130009B0703D009E008C9121F08C0042AFAD29D
:1001400003E00B780370401C491C521EF9D2704723
:10015000D2B201E00270401C491EFBD2704700225F
:10016000F6E710B513460A4604461946FFF7F0FFB6
:10017000204610BD064C0125064E05E0E36807CC7D
:100180002B430C3C98471034B442F7D3FFF79CFF45
:10019000C0070001D0070001F7B5D4B004460E46F1
:1001A00000205390052052900025002700BFEFF358
:1001B00010800090FF21453101A8FFF7D0FF00F02B
:1001C000F1F905462448854218D1012000038442F4
:1001D00002D1002053902AE001204003844202D142
:1001E0004011539023E003200003844203D10120F7
:1001F000400253901BE0529857B0F0BD174885421B
:1002000013D101200003844201D153900FE001205B
:100210004003844201D1539009E00320000384424B
:1002200001D1539003E05298E6E75298E4E705AF16
:100230000137FF2241320A4901A8FFF777FF012069
:1002400000F04FF93146569A5398B84752900098AB
:1002500000F047F95298CFE7C440130085601300BF
:10026000E8050001F1B58AB0002009907D20C000AA
:1002700008900125AD020027002007907F200690FE
:1002800040240026002005900390200102900020C9
:1002900001903E490A98884206D83D4800686102AC
:1002A00088433B49086006E0394800680121C903DA
:1002B0000843374908607D21C9000A98FFF720FFED
:1002C0007D21C9000090FFF71BFF450100BF3048AA
:1002D00000687F21090288430190200201990843A8
:1002E0002B4908600520FFF7F9FE10E00120FFF719
:1002F000F5FE2748406B02210840002800D007E0A7
:100300000598411C05910899884200D900E0EDE765
:1003100000BF1F48C06B86B2AE4201D9771B00E018
:10032000AF1B0298874203D2E0B20390B8B20290AA
:10033000AE4201D3069400E007940699079840184E
:10034000C005000E04900498A04200D103E0049C74
:1003500009988742BBD800BF0D4800687F21090279
:1003600088430190039800020199084308490860F6
:100370000846406840084000486000BF04484068A4
:10038000042108400028F9D10BB0F0BD0090D00343
:100390000010024010B53E48C0690121090708431A
:1003A0003B49C861812000063A4908633A484861E0
:1003B0003A4808623A48006803218903884338496B
:1003C00008603421374800F073F836480069401C53
:1003D000002803D033480069002817D12C48406812
:1003E0000121090408432A4948600846406807215A
:1003F00009028843264948600846406809150843B1
:10040000234948602848FFF72DFF3FE021488069D5
:100410004409640123480078C006C00E04431D4807
:1004200084611B4800680121C9038843184908609A
:10043000084600687F21090288430446194800697C
:10044000000220431249086008464068012109045F
:1004500008430F494860084640680721090288435D
:100460000B49486008464068091508430849486038
:100470000846006A0D490840054908620846006AB6
:100480000849C968090208430149086210BD000013
:1004900000100240007000400F0800001800020029
:1004A00000100140004000200090D003FF00F8FF42
:1004B00070B504460D462A46214601200003FFF789
:1004C0006BFE70BD02E008C8121F08C1002AFAD1F5
:1004D00070477047002001E001C1121F002AFBD1C4
:1004E000704780F31088704730B502460B460021F4
:1004F000C94312E01078521C414000240BE0480828
:10050000CD07ED0F002D01D0074D00E0002568401C
:100510000146601CC4B2082CF1DB18465B1E0028A3
:10052000E8D1C84330BD00002083B8ED0446012067
:10053000C007204305490863206880F3088800BF8E
:1005400062B66068804700BFFEE7000000700040B0
:10055000114C124D1249206888421AD12821204698
:10056000FFF7C2FFA16A884213D16168022902D154
:100570002146183101E0214608310846074A016842
:10058000914205D32122D2040168914200D205682C
:1005900000BF2846FFF7CAFF0040000100800001AD
:1005A00011C011CA70B5D2B00024002500BFEFF30E
:1005B00010800646FF21453101A8FFF7D0FD01ACB0
:1005C00001349822074901A8FFF7B0FD0120FFF789
:1005D00088FFA04705463046FFF783FF284652B004
:1005E00070BD00002807000140BA7047C0BA7047CC
:1005F0000138FDD170470000F7B50325AD06286A24
:1006000082B016460C46400840002862286A022143
:1006100008432862286A8007FCD4662068600127A6
:100620002F61A86AC005FCD5992068602F61A86A6F
:10063000C005FCD5FF209130FFF7DAFFFF2301331F
:10064000AB626846EF60352169602F61A96AC90510
:10065000FCD5AB62A969EF60C9B205226A602F615F
:10066000AA6AD205FCD5AB62AA690902D2B21143CB
:100670000180C80702D0032005B0F0BDAB626869F5
:10068000FF210831884368616869C91E08436861B1
:1006900002980002483068600820A860EE602F6170
:1006A000A86AC005FCD5FF200130A8620023F61C13
:1006B000B0080ED0B2081148006899006054060ACC
:1006C00009194E70060C000E8E705B1CC8709A42A1
:1006D000F1D8FF200130A8626869FF210831884302
:1006E0006861686938436861286A80088000286208
:1006F000286A38432862002005B0F0BD8000000C55
:10070000032080064169FF2208329143416142691A
:1007100001210A434261026A920892000262026A5F
:100720000A43026270470000002003218906096A1B
:10073000490849000322920611621146096A022201
:10074000114303229206116200BF03218906096A40
:10075000022211400229F8D0D101032292069162AF
:100760000321D1609F2151600121116100BF03214C
:100770008906896AFF22013211409142F7D1032292
:1007800092069162114688694969FF2208329143B5
:100790000322920651611146496901221143032245
:1007A000920651611146096A890889001162114651
:1007B000096A012211430322920611627047000068
:1007C000D00700010040002038080000D4040001D8
:1040000011C011CA010000000080000110740000FE
:10401000F077394C000000000000000000000000B4
:0C402000000000000000000016B76EF465
:1080000040B000205D8100016581000167810001B1
:108010000000000000000000000000000000000060
:10802000000000000000000000000000D58E0001EC
:1080300000000000000000001B810001D98E00013B
:108040006F8100016F8100016F8100016F8100016C
:108050006F8100016F8100016F8100016F8100015C
:108060006F8100016F8100016F8100013587000180
:108070006F8100016F8100016F8100016F8100013C
:108080006F8100016F8100016F8100016F8100012C
:108090006F8100016F8100016F8100016F8100011C
:1080A0006F8100016F8100016F8100016F8100010C
:1080B000B19000016F8100016F8100016F810001AB
:1080C0000348854600F092FA0048004789BA00014B
:1080D00040B0002040BA7047C0BA70470138FDD1A7
:1080E00070470000084B19680868203080F3098841
:1080F000022080F31488BFF36F8F3FBCAE4608BCEC
:1081000004BC62B61847000050470020EFF310800F
:1081100072B6704780F310887047EFF309800E4BFA
:108120001A6820381060F0C044464D4656465F46F7
:10813000F0C008B572B605F057FE62B60CBC116807
:1081400008681030F0C8A046A946B246BB4680F386
:1081500009882038F0C81847504700200448804755
:1081600004480047FEE7FEE7FEE7FEE7FEE7FEE71E
:10817000318F0001C180000130B50B46014600205F
:108180002022012409E00D46D5409D4205D31D461D
:108190009540491B2546954040191546521E002D15
:1081A000F1DC30BD70B500242546002801DA012439
:1081B0004042002901DA01254942FFF7DDFFAC42C8
:1081C00000D04042002C00D0494270BDF0B51FB431
:1081D0000646002082B005464024019100901BE035
:1081E000019922460F46304600F090F9049A059B0B
:1081F000801A994110D310461946224600F076F9AC
:10820000361A8F410197224601200021009F00F07D
:108210006DF938184D4100902046641E0028DFDCBF
:10822000019B00982946324607B0F0BD0549064A31
:1082300008685043054A80180860400870470149A3
:1082400008607047A84700206D4EC64139300000D5
:1082500003460B439B0703D009E008C9121F08C05F
:10826000042AFAD203E00B780370401C491C521E0A
:10827000F9D27047D2B201E00270401C491EFBD215
:1082800070470022F6E710B513460A460446194621
:10829000FFF7F0FF204610BD30B50446002003462E
:1082A00000E05B1C934203D2E05CCD5C401BF8D045
:1082B00030BD0000F0B51FB488B00B9909980024B8
:1082C00048400999C00F490049080991C0070B9916
:1082D0000090490049080B9109990898A64608435F
:1082E0001CD00B990A98084318D009980124400023
:1082F000420D4800410D099824050003000B20435E
:1083000009900B980003000B20430B9050181C4958
:108310004018002201901446104605E00020014656
:108320000DB0F0BD032801DA034600E003239C46AC
:10833000C11A0AAE0AE05F0008ADED5B4F00F75BC3
:108340007D430027AA187C41491C5B1E6145F2DD74
:10835000410004AB5A522104120C0A43240C401C65
:108360000828DFDB01980290009970460191009087
:10837000059B049A0799069800F0E6F8D0E70000FC
:108380000DFCFFFFF0B50C465C4085B0E40FE40740
:1083900003944C000026640859009446490802469C
:1083A0000296224321D062460A431ED06200570D36
:1083B0004A000E032303550D012402462C492405CF
:1083C000781B1B0B360B4018234326436146009055
:1083D0001C46501AB44103D30098401C009002E0A0
:1083E000921800985B41002803DA0020014605B08E
:1083F000F0BD0020012109050746864611E06446CC
:108400001D46141BB54106D36546521BB341744645
:1084100007430C43A646CD07400849082843921855
:108420005B4105460D43EAD11046184313D0604620
:10843000194650407140084306D06046101AB341B7
:1084400006D20122002306E000220123DB0702E01E
:108450000122D2435310009874460105381C614133
:10846000029C039D0019694100F061F8BFE700001C
:10847000FD0300000EB505490291002100910A4656
:108480000B46019100F060F803B000BD330400001A
:108490000EB5054A0292002200921346019200F0A6
:1084A00053F803B000BD0000330400004A00090384
:1084B0000123090B1B0519430A4B10B5520D9A42B3
:1084C00002DA0020014610BD064B34339A4203DC29
:1084D0009A1A00F01BF810BD034BD21800F006F8F2
:1084E00010BD0000FF030000CDFBFFFF10B5202AE8
:1084F00004DB0146203A9140002010BD914020232A
:108500009C1A0346E3401943904010BD10B5202A41
:1085100004DB0846203AD040002110BD0B46D34072
:10852000D0402024A21A91400843194610BD10B52E
:10853000002B08DA0024401C614192185B411A4369
:1085400001D14008400010BDF0B51FB482B005460F
:108550000C0003D0084600F045FE02E000F042FEA9
:1085600020300246009021462846FFF7BFFF049BBB
:10857000059A04460F4618431143084314D0184681
:1085800010431BD0009840210A1A18460599FFF79E
:10859000BDFF05460E46009A05990498FFF7A6FF11
:1085A000084305D0012004E02046394607B0F0BD5D
:1085B0000020C11705430E432C43374300990E9802
:1085C0006305401A7905E40A00220C43FD0A0A30CB
:1085D00002D500200146E9E70105101969410C9C0C
:1085E0000D9D00196941FFF7A2FFDFE7064C012549
:1085F000064E05E0E36807CC2B430C3C984710344B
:10860000B442F7D3FFF760FDE8ED000108EE00018A
:1086100070B58C180578401C6B075B0F01D103788F
:10862000401C2A1106D10278401C03E006780E7027
:10863000401C491C5B1EF9D12B0705D40023521E98
:108640000DD40B70491CFAE70378401CCB1A921C1E
:1086500003E01D780D70491C5B1C521EF9D5A14228
:10866000D8D3002070BD000003B40148019001BDC3
:10867000232A000003B40148019001BD6D5600009B
:1086800003B40148019001BD6560000003B40148D6
:10869000019001BDAF7F000003B40148019001BD0E
:1086A000B551000003B40148019001BDD37E000024
:1086B00003B40148019001BD697E000003B4014884
:1086C000019001BDC37F000003B40148019001BDCA
:1086D000E954000003B40148019001BD995700001E
:1086E00003B40148019001BDED57000003B40148F7
:1086F000019001BD7184000003B40148019001BDE7
:108700001D7C000003B40148019001BDAB52000084
:1087100003B40148019001BDF58F000003B4014886
:10872000019001BDB143000003B40148019001BDB7
:108730008529000010B5164C0220214600F0CFF824
:1087400000280BD0134A0020107003221146124853
:108750000FF442D22146022000F020F821462020CA
:1087600000F0BDF8002805D02146202000F016F8C2
:1087700005F00CFA2146402000F0B1F8002805D0A1
:108780002146402000F00AF805F000FA10BD000074
:108790000000024038470020120F00004860704778
:1087A000002A026801D00A4300E08A430260704751
:1087B00030B51C4C8BB0204600F03EF81A4D01231A
:1087C00022462946022000F0B1F80122022120466B
:1087D000FFF7E6FF154C204600F02EF80123224655
:1087E0002946032000F0A2F8012206212046FFF7C7
:1087F000D7FF0F480090A1150E480391019020214A
:108800000020089180210591049003210290090322
:108810000690079009910A906946204600F066F894
:108820000BB030BD08000240000002401C000240B6
:1088300004380140804E002001681A4A114001604E
:108840000021016041608160C160174A1749904270
:1088500004D148680F22104348607047144A904280
:1088600004D14868F022104348607047114A904292
:1088700005D148680F2212021043486070470E4A23
:10888000904205D148680F22120310434860704798
:108890000A4A9042FBD148680F22120410434860F4
:1088A00070470000FEFF0000080002400000024088
:1088B0001C000240300002404400024058000240C8
:1088C0000029016802D00122114301E0014A114050
:1088D00001607047FEFF0000406880B270470246AA
:1088E00009680020114200D00120704730B40368AD
:1088F0000D4A0C6A13408A684D6922430C692C4367
:1089000022438C692243CC6922434C6A22438C6AFD
:1089100022431A430260CA6842600A68826049685A
:10892000C16030BC704700000F80FFFF002B01D0FA
:1089300010617047002010617047000001494861D4
:108940007047000000040140054B002219685B6974
:108950000140034202D0002900D001221046704796
:108960000004014010B4837919490268002B28D013
:108970000B6893430B604A6803689A434A60027924
:10898000521813680468234313608A6803689A4383
:108990008A60CA6803689A43CA604279102A06D07E
:1089A00051180A68006802430A6010BC70478A6860
:1089B00003681A438A60CA6800680243CA6010BC30
:1089C00070470079401801689143016010BC7047FE
:1089D000000401400B680022002B56D0F0B40124A3
:1089E0000B68944023424AD04B68022B01D0122BD3
:1089F00016D113070AD5456A5307DB0E0F269E4092
:108A0000B5434E699E402E43466209E0056A53070E
:108A1000DB0E0F269E40B5434E699E402E430662F4
:108A20004B68012B05D0112B03D0022B01D0122B48
:108A300006D14568DB06DB0FA54393402B4343601B
:108A40000568530003279F400E79BD43B607B60F54
:108A50009E402E430660C5688E68BD439E402E43EF
:108A6000C66085680126A543CC6894402C43846089
:108A7000C46A9E400D69B4439D402543C5620B689E
:108A8000521CD340ABD1F0BC704770470549016020
:108A9000002242600F218260416101210261C160B8
:108AA00070470000FF3F000081627047816170479E
:108AB00042694A40426170470180704705498842D7
:108AC00007D10548026A01040A430262026A8A4326
:108AD00002627047004800400010024002461288BF
:108AE00000200A4200D0012070470000F0B5054682
:108AF000008989B00E4600242C49F2880840B188CC
:108B00007389114332891A4311430143298128484B
:108B100085420AD1002000F0D3F901218906CF1245
:108B2000884206D02349884203D001A800F08EF97C
:108B3000039F31683846FFF71FFB0A2808D8012237
:108B4000298992038904890C29812989114304E028
:108B500029898904890C298129892981A881366874
:108B600038463146FFF708FB08461349484331466B
:108B7000FFF702FB00260790009007990690401827
:108B80000D490090FFF7F8FA07460B490698FFF7E2
:108B9000F3FA874202D00120A0400643641C082C4F
:108BA00001D20098E9E72E7509B0F0BDF47000001D
:108BB00000480040200000041027000001747047A6
:108BC00010B5FFF775FF10BD30B505460E4887B0EC
:108BD0000C46854202D10121042004E00B48854265
:108BE00010D10121082000F019F90948844209D860
:108BF0006846FFF74BFF0120019069460094284624
:108C0000FFF7E8FE07B030BD00080140000C01404E
:108C1000FF3F000010B5FFF747FF10BD10B5FFF78D
:108C200045FF10BD10B400214156FF23CAB2920780
:108C3000D40E4278A3409207120EA24000290BDA0C
:108C40000907090F08398C081049A4006118CC697C
:108C50009C431443CC6107E08C080D49A4006118C3
:108C60000C689C4314430C60827801210078002A30
:108C700004D0C006C00E8140064803E0C006C00E06
:108C800081400548016010BC7047000000ED00E025
:108C900000E400E000E100E080E100E0F7B5FFB0B3
:108CA00004460025A5B00520EFF31087FF210090B2
:108CB000453102A8FFF7E5FAEFF31086FF214531B1
:108CC00053A8FFF7DEFA53A80130019098222249F9
:108CD00053A8FFF7BDFA012080F310880198804760
:108CE00086F3108801221D49120303265300360320
:108CF00088420AD194421AD09C4201D1151116E043
:108D0000B44210D101256D0211E0154988420AD103
:108D1000944201D115460AE09C4201D11D4606E06D
:108D20003546AC4203D000987FB028B0F0BD06AC09
:108D3000FF22013441320B4902A8FFF789FA0120D2
:108D400080F310882846A69AA599A04787F3108833
:108D50007FB028B0F0BD0000F0E20001C440130075
:108D600085601300B0E1000110B5EFF3108401211C
:108D700081F31088FF2109064018034909688847D4
:108D800084F3108810BD00000440002010B508488E
:108D9000064901600749416007498160C922920084
:108DA00006490748FFF754FA10BD0000814800202B
:108DB0000440002015490020E947002094E3000109
:108DC000E047002010B5EFF31084012383F31088EF
:108DD000FF231B06C018034B5B68984784F3108879
:108DE00010BD000004400020002808D10448026A99
:108DF00001239B069A430262026A0A430262704799
:108E000000100240044A0029516901D0014300E0EA
:108E1000814351617047000000100240044A00295C
:108E2000916901D0014300E08143916170470000E6
:108E3000001002400449CA030128086A02D0904386
:108E4000086270471043FBE70010024030B4164A36
:108E5000516804231940154B01D0042901D0036047
:108E600001E0134901605168124B8906890F5B5C70
:108E70000168D940416053680F4C5B055B0FE35CB0
:108E80000D46DD40856053689B045B0FE35CD94071
:108E9000C160D16AC90601D5084901E07D21C90335
:108EA000016130BC70470000001002400090D00308
:108EB0000048E80188E300018CE3000100093D005F
:108EC0000248006A02490840704700000010024052
:108ED000200000047047000010B5FFF717F90446A2
:108EE00005F098F8002803D00120034900074860E6
:108EF0002046FFF70FF910BD00ED00E010B50A4C59
:108F00002069411C01D000280AD1012006493422E1
:108F10000003FFF7C3FE2069411C03D0002801D0E5
:108F2000024810BD002010BDAC470020D5470020EE
:108F3000F0B5564C85B0E06921040843E06181201A
:108F4000534D0006286353486861534828625348CC
:108F50000322016892039143016051493422801435
:108F6000FFF79CFE4E4B4F4E18694F4F411C29D0C6
:108F7000002827D0A9691A7849094901D206D20EDA
:108F80000A43AA612168EA139143216021687F2284
:108F90001202914300020843206060683043606021
:108FA0006068B84360606068211508436060206AAB
:108FB0003E4908402062206AD968090208432062BD
:108FC00005B0F0BD61682046314361606168B94316
:108FD000616061680127BF0239436160002104912B
:108FE0007D21C9000391002100917F2140240025AB
:108FF00002950191026861028A4302600E112349C1
:1090000008687F2212029043220202430A60052070
:10901000FFF764F80120FFF761F81C48406B8007F8
:1090200004D4284603996D1C8842F3D91748C06BB5
:1090300080B2B04201D9811B00E0311AB94202D29C
:10904000E2B28FB20292B04201D3019400E00094E8
:10905000019A00988018C005000EA04203D0044673
:1090600004988142CBD8094801687F2212029143BB
:10907000029A12020A4302604168490849004160AD
:1090800041684907FCD405B0F0BD00000010024063
:10909000007000400F08000018000200001001409E
:1090A000AC4700200000010000070000FF00F8FFAF
:1090B00010B5054C1021204600F038F8002802D0E9
:1090C000A08804F063FD10BD0038014010B40B0609
:1090D000CC065B0FE40E0121A140012B07D0022B2F
:1090E00007D01430002A026805D00A4304E00C308F
:1090F000F8E71030F6E78A43026010BC70470000C2
:109100000029818903D001225203114301E0024A60
:109110001140818170470000FFDF0000002A828A31
:1091200001D00A4300E08A438282704702461288D7
:1091300000200A4200D001207047000070B50446AC
:10914000008A86B00D461B490840E9880143218208
:10915000A08919492A890840A98811436A890243CC
:109160001143A181A08A15490840A9890143A18220
:109170006846FFF76BFE1248844201D1039800E075
:1091800002982968192289005043FEF7F5FF064628
:109190006421FEF7F1FF0501280964214843301AD4
:1091A00000013230FEF7E8FF0007000F284320815E
:1091B00006B070BDFFCF0000F3E90000FFFC000027
:1091C000003801400FB410B503A9044B044A0298BB
:1091D00000F020F810BC08BC04B0184721A500011D
:1091E000C40100202021020C01D010211046020AE7
:1091F00001D010460839020901D01046091F820823
:1092000001D01046891E420801D0881E7047081AF6
:1092100070470000FFB591B00F460546002606E0F6
:1092200025280AD0149A139990476D1C761C28782B
:109230000028F5D1304615B0F0BD0024009401217E
:10924000F34A029400E004436D1C2B780846203B4F
:1092500098401042F7D128782A280ED00221287889
:109260000246303A092A15D8009A0A235A43303A5E
:1092700080180C436D1C0090F1E701CF009000288E
:1092800005DA012040030443009840420090022088
:1092900004436D1C28782E2815D1042004436878D7
:1092A0006D1C2A280AD101CF6D1C02900BE0029997
:1092B0000A225143303940186D1C0290287801462B
:1092C00030390929F3D928786C2810D006DC4C28CD
:1092D0001AD068280ED06A2817D104E0742813D059
:1092E0007A2812D110E00120400504430CE001214E
:1092F000090501E0032109050C436978814203D186
:109300000120000524186D1C6D1C287803906E2820
:109310001ED00CDC632831D004DC00288AD0582809
:1093200011D1B2E064287BD069280CD178E0732891
:109330002DD004DC6F2870D0702804D1A7E07528E8
:109340006CD078286BD0149A13999047761C62E001
:109350006002400F022807D003280AD0042838688A
:109360000AD006603F1D56E03868F117066041607C
:10937000F8E738680680F5E70670F3E7387869465D
:1093800008740020487404A80390012003E03868A2
:1093900003900020C0433F1D61070FD5002101E06D
:1093A0000199491C029A0191914213DA8142F7DB3B
:1093B000019A0399895C0029F2D10BE0002101E0B8
:1093C0000199491C01918142FADB019A0399895C58
:1093D0000029F5D101990098139A401A009021466E
:1093E000149B00F03BF901998019461807E0039897
:1093F00003990078491C0391149A13999047019896
:10940000401E0190401CF2D12146149B139A0098F3
:1094100000F014F986196D1C09E741E033E034E0EF
:109420000A200021049005916002410F022905D015
:1094300001CFC2179446032905D007E0FF1DFF089E
:10944000FF0003CF06E000B2C2179446042902D100
:1094500040B2C1178C4600226146944506DA0A469E
:109460000021404291418C462D2102E0210504D586
:109470002B216A461176012103E0E10701D020216A
:10948000F7E7019154E00A200BE0102009E01020DA
:10949000049000210420044308200591029003E079
:1094A00008200021059104906002410F022905D097
:1094B00001CF00229446032906D006E0FF1DFF08D5
:1094C000FF0003CF8C4603E080B2042900D1C0B274
:1094D0000021019121072BD50399702906D0049A08
:1094E0001021059B4A401A4305D00EE040216A46F0
:1094F0001176012108E06146014306D030216A4619
:1095000011760399517602210191049A0821059B55
:109510004A401A430CD16146014301D1610707D586
:1095200030216A461176012101910299491E02916A
:109530000399582904D037A103910FA90F910DE089
:1095400039A1F9E76146059B049AFEF73FFE039BAC
:109550008C469B5C0F9A521E0F921370614601431A
:10956000F0D10F9807A9081A20300390600704D59E
:10957000012000048443029801E001200290039935
:10958000884201DD401A00E0002041180290019855
:1095900009180098401A0090E00306D42146149B55
:1095A000139A009800F05AF886190020049008E0F9
:1095B00006A9085C149A139990470498401C761CDD
:1095C000049001998842F3DBE0030CD52146149BFB
:1095D000139A009800F042F8861904E0149A30209B
:1095E00013999047761C0299481E02900029F5DCD9
:1095F00008E00F980F990078491C0F91149A13995D
:109600009047761C0399481E03900029F1DCFBE685
:109610000928010030313233343536373839616248
:10962000636465660000000030313233343536370C
:10963000383941424344454600000000F8B504462D
:1096400000251E461746880404D405E0394620202C
:10965000B0476D1C641EF9D52846F8BDFFB5044619
:10966000002581B01E46C80301D5302700E0202721
:10967000880404D505E038460399B0476D1C641E84
:10968000F9D5284605B0F0BD00B599B0602168460F
:10969000FEF7F7FD042008AAD07012A00068019020
:1096A0000B2010AAD070024610A109A8FEF7D0FD29
:1096B000002010AA107101215171D0719171907325
:1096C0001175D082A02010839176B4209083192048
:1096D000C001D08308480090684602F0A9FB19B089
:1096E00000BD000003160A18000000000AFFFFFF7B
:1096F0004E6174696F6E7300FD9600017047000043
:1097000010B58CB000240094019402940394049446
:10971000059406940794089409940A94FFF7EEFBC5
:10972000002804D0014601A8FEF79EFF07E012A022
:1097300001886A4691804188D1808088108169467D
:10974000CC704C810A20887012220A7303A80CA1E5
:109750000130FEF77DFD0C206946088418204884FE
:10976000FF208C84F530C8840A480885684602F0DA
:1097700021FC0CB010BD000001020304050600002E
:1097800043414949432D4D434D2D32303236303916
:10979000303200008813000000B583B00D490091FD
:1097A0000D4900200191029069460872684602F056
:1097B000EBFCFFF7A5FF00F045F8FFF765FF074852
:1097C00002F0A2FA064802F09FFA02F055FB03B03D
:1097D00000BD0000E597000199A00001719900010A
:1097E000999B000170B50178012911D000250E4E1A
:1097F0000E4C022910D0032909D102F03DFB0020B4
:1098000000F040FB40213046FFF704FA257070BDA0
:1098100007A0FFF7D7FC70BD012000F033FB40210B
:109820003046FFF7FBF9F1E7000801403747002019
:109830004150505F424C455F4F535F524541445940
:109840000D0A000000B587B0002001900090039041
:1098500004906A46069010730C490291052191709C
:10986000032313701023D3705070107101235371B0
:1098700090715073064805907D209173000110820D
:10988000104603F0B3F907B000BD000040E201004C
:1098900000B0030110B5024802F0E4FE002010BD44
:1098A000F44D00202F48007900285AD1F8B56D20DA
:1098B0002C230322072140010EF43ED1A0210446AF
:1098C000017029480027C178617027710321E18068
:1098D0006772012666710721244D2177A979617786
:1098E000687B002803D0E780032060710EE0E879F0
:1098F00000280BD0A879022800D166772671E6806F
:109900002046A9792030417086700770154880790B
:10991000022804D0032815D004281BD116E003F038
:1099200057F900280BD00520E0806771688A6061D4
:10993000688AA06120460A3002F01EFF0AE0094949
:1099400003208871288B6061288B02E0E88B6061BE
:10995000E88BA06103480671467120460EF428D1B9
:10996000F8BD7047504D0020D44D0020404E0020DF
:1099700010B584B00A230322072110480EF4DCD06E
:109980001B21017000214170142444800322828035
:10999000C1800B4A02810EF40BD16846048009484D
:1099A0000190684602F0B8FB6846048106480390BF
:1099B00002A803F06BFA04B010BD00001B0D0000FC
:1099C000FF01000014ED0001E5A20001FFB585B024
:1099D000054602A800901C462846069903F050F957
:1099E0006846007A002866D006980090280A334A14
:1099F000019403900E2826D03148002401780029D4
:109A000051D92F48E1000818828803998A4240D131
:109A1000009A81689646019A284694460A79120669
:109A2000120E36D00968254BD700083FCE1937886B
:109A30007668BFB2874201D09F4226D16346032297
:109A40007146B04725E01F49681809282BD80098AF
:109A50001D49844608792E4600062346000E1ED076
:109A6000C4000F68083C3C1927886468BFB2B7423D
:109A700001D0974204D1032261462846A0470EE058
:109A8000401E0006000EEBD109E0521E1206120E17
:109A9000CAD10B48641C0078E4B2A042B1D8684631
:109AA000007A002807D00948426C002A02D02846D4
:109AB00006999047002009B0F0BD0000FFFF0000AC
:109AC000FC4C0020EEF1FFFF18E80001504D002093
:109AD00010B502F08DFD04480169002901D0042071
:109AE0008847002010BD0000604E002070B5224C59
:109AF000606B224DC00722D0A06B21497E220968ED
:109B00005143401A2988491E29804B21C900401819
:109B10001C49884213D300202880206A4008400056
:109B20002062194908680204930F184A01D0904333
:109B300000E0104308601648407F02F0ABFA298825
:109B400001200029216B07D0014321630522032155
:109B500010480EF4B3D20DE0FF22120291432163AC
:109B6000216B0522920211432163216B0143216382
:109B700003F07CF8002070BD001002403447002044
:109B80008C000020B10400000010014000C0000063
:109B9000B04D0020010F000010B584B01423032243
:109BA000072112480DF4C8D71B2101700021417014
:109BB0004724448003228280C1800D4AC2600D4A3E
:109BC0000261072202720DF4F3D7684604800A4846
:109BD0000190684602F0A0FA6846048107480390A5
:109BE00002A803F053F904B010BD00001B0D0000E3
:109BF00034ED000124ED00011CED00013DD5000114
:109C000000207047F8B5184D184FE879002801D0AA
:109C10002E7B00E0FE780322331D072114480DF44B
:109C20008BD7A921044601701248C17861700021C8
:109C30006180E8791049002803D02A7B896C201DB7
:109C400002E0FA78201D091DFEF702FB6088022160
:109C50008019608007480279062A00D0017141719D
:109C600020460DF4A5D7F8BD404E0020204E002020
:109C7000A60D0000504D0020004E0020F8B51F2614
:109C800023230322072128480DF456D70446AA208F
:109C9000264F2070F878264D6070E8786080EA786A
:109CA0002449201DFEF7D4FA6288B01AC1B2201DE3
:109CB0001018214A0326032910D92B79002B0DD027
:109CC0000670192343705389091F1B0AC370937AC6
:109CD00083706388C9B21B1D6380001D02291AD9D5
:109CE0006B79002B17D0137B891E8B4200D219464B
:109CF000CDB2691C0170117BA94201D1092100E09C
:109D0000082141702A460D49801CFEF7A1FA60889F
:109D1000AD1C401960803879062800D03E717E71F4
:109D200020460DF445D7F8BDA60D0000504D00208B
:109D3000404E0020244E0020D44D0020E14D002054
:109D400070B53A230322072116480DF4F5D6A42155
:109D5000154D04460170E8786070A9791348002217
:109D6000022910D0032913D0042916D06280227151
:109D7000807901F091FD052028710420687120464A
:109D80000DF416D770BD018A642359436180EEE754
:109D9000C18A642359436180E9E7818B6423594375
:109DA0006180E4E7A10D0000504D0020404E0020EE
:109DB00070B58AB001210820FFF730F8012188032F
:109DC000FFF72CF801210846FFF71CF86846FEF75C
:109DD0005DFE402000900220254D0424019069463C
:109DE00005942846FEF7F6FD80210594009169460A
:109DF0002846FEF7EFFDFEF7DBFC0B2001241D4D8E
:109E0000E10229606946087003264E708C7068462E
:109E1000FEF708FF1C2021072960694608704E7074
:109E20008C706846FEF7FEFEE1204002069000209E
:109E300069468883C883088488840C2048840E4C33
:109E400006A92046FFF77AF901220C492046FFF7C0
:109E50003DF90122C0212046FFF760F901210848A1
:109E6000FEF72EFD01212046FFF74AF90AB070BD2A
:109E7000000C014080E100E00038014024040000B3
:109E80001C00024010B5002486B001281BD002F04F
:109E9000EDFE00211248FFF733F900211148FEF7CB
:109EA0000FFD00211048FEF70BFD6846FEF7EEFDA2
:109EB000C020009003200190694605940B48FEF7EE
:109EC00089FD06B010BD02F0C5FE094884804461DA
:109ED0000461C4608460FFF76BFF06B010BD000032
:109EE000003801401C00024008000240000C014004
:109EF00038470020F8B5234F0C00064638D0F968E3
:109F0000B868884218D37D21C9000D1AA54200D92E
:109F100025461D492A4608183146FEF799F9601B67
:109F200084B2B8687D2176194019C900FEF724F97A
:109F3000B960002CE3D11BE00D1A6D1EA54200D9BB
:109F4000254611492A4608183146FEF781F9601B5B
:109F500084B2B8687D214019C900FEF70DF9B960D7
:109F6000002C05D00A46214608A0FB68FFF72AF915
:109F70007878002804D10A22032108480EF49ED0E4
:109F8000E0B2F8BD38470020804F0020463A2564F3
:109F90002C25642C25640D0A0000000007470000F2
:109FA000F8B5064624480C0047693ED022490869A6
:109FB000B8421AD37D22D200151AA54200D92546EF
:109FC0001E4A314610182A46FEF742F9601B84B239
:109FD00019487D21006976194019C900FEF7CCF8AF
:109FE0001548002C0161E1D11FE013490A69BD1A2F
:109FF0006D1EA54200D92546104A314610182A4642
:10A00000FEF726F9601B84B20B487D210069C90068
:10A010004019FEF7B1F80848002C016105D00A4646
:10A020003B46214606A0FFF7CDF83222032108481F
:10A030000EF444D0E0B2F8BD384700206853002049
:10A04000463A25642C25642C25640D0A0000000086
:10A05000120F000070B50E4D0E4869692C6940184A
:10A06000A14207D2611A89B203F0BAFD012800D1DA
:10A070006C6170BDA142FCD97D22D200511A89B217
:10A0800003F0AEFD0128F4D10020686170BD00002E
:10A090003847002068530020034910B5C84201D159
:10A0A000FFF7D8FF10BD0000EEF0FFFFFFB50F4631
:10A0B00083B000210091019116466946FEF7DAFA55
:10A0C000040030D10521C9026846FEF7D9FA0028FC
:10A0D00028D121496846FEF7D3FA002822D11F492A
:10A0E0006846FEF7CDFA00281CD11D496846FEF7E8
:10A0F000C7FA002816D1292109026846FEF7C0FADE
:10A1000000280FD117496846FEF7BAFA002809D18E
:10A1100015496846FEF7B4FA002803D100988088F4
:10A12000C10B03D00624204607B0F0BD00050099FE
:10A13000000D0D186888B04200D207242988B8198C
:10A14000884201D90D24EEE7A8193A46001D069968
:10A15000FEF77EF86F80E6E7012800000328000084
:10A1600002280000022900000329000021F418D170
:10A17000012003F0F1FDF9E702468B880020022B55
:10A1800001D00D207047C988002A05D00029F9D0D8
:10A190000129F7D0812070470029FCD00229F9D18C
:10A1A000704702460020802901D98D207047062A79
:10A1B00006D0072A07D0082AF8D10729F5D1704719
:10A1C0000829F2D170470629EFD3704770477047CE
:10A1D00070B5C46805466068002803D000200028D8
:10A1E00002D00CE00120FAE7201DFEF74FFA0DF433
:10A1F00093D36068002808D000200028F4D0002005
:10A20000E86020460DF488D370BD0120F5E730B436
:10A210000446A2890920521C93B2E48900222546F3
:10A22000D540ED0707D05D1C8D4202D130BC1046F1
:10A2300070479B1C9BB2521CD2B2092AEFD330BC90
:10A2400070470000FFB585B00E9D04462F880120A1
:10A250001E4600213A46CA40D20704D04B000322D2
:10A260005B1C9A401043491CC9B20929F2D30490DF
:10A2700030461E210840218A184A0023019100938C
:10A2800002920390132304AA15490698FEF704FAD4
:10A29000009000281FD1012114200DF4C7D30746D8
:10A2A000E06006980188B9812988F981F00701D01A
:10A2B0000120C003079908433880208A7880142041
:10A2C0006082204600F060F8381DFEF7EBF9208A26
:10A2D00000210DF401D5009809B0F0BDD8E60001C9
:10A2E0000A1800000048704770E70001FFB50878C1
:10A2F00081B00C46092836D2142002F093FD07469F
:10A30000217800F0EFF800282BD061782078FFF753
:10A3100048FF060028D17D68002D0ED020782979CD
:10A32000814207D12946381DFEF7C2F928460DF4AF
:10A33000F3D202E02D68002DF1D1607801210830C0
:10A340000DF474D3054620782871607868716278BE
:10A35000A11CA81DFDF77CFF2946381DFEF7AEF9AC
:10A3600002E0822600E0812602230648039A04992F
:10A370000DF4E2D32178017046700DF419D4002059
:10A3800005B0F0BD0114000010B50446142002F021
:10A3900049FD044921600321618112306060012080
:10A3A000208110BD80E70001F8B517460C46104625
:10A3B0000DF480D4012831D1142002F033FD05467C
:10A3C000017C00F08FF80646297C227814489142DF
:10A3D00014D1697C637809023A46891D9B1D0DF4EE
:10A3E000ABD30546068000202871607868806278CB
:10A3F000A11C681DFDF72CFF284609E0697C062397
:10A4000009023A46891D0DF497D306808021017117
:10A410000DF4CED3002138460DF45ED40020F8BDF3
:10A42000140C0000F8B50F4600240978184625469C
:10A4300009291DD20B007B441B79DB189F440407BC
:10A44000101313130A160D00052414A510E00A2496
:10A4500014A50DE0082416A50AE0072417A507E0B7
:10A460000A2418A504E0052419A501E006241AA56C
:10A470000146A31C1A480DF45FD3064638783070A5
:10A480007470002C04D022462946B01CFDF7E0FE73
:10A4900030460DF48DD30020F8BD00004E53494ED8
:10A4A000470000004E532D424C452D312E30000008
:10A4B000123456FFFE9ABCDE00000000025E04402B
:10A4C00000000300312E302E302E302D4C45000080
:10A4D000312E302E30000000FFEEDDCCBBAA000094
:10A4E0000314000010B48289C489521C93B2002264
:10A4F0002046D040C00706D0914202D15B1C9BB2DF
:10A5000005E09B1C9BB2521C52B2092AF0DB092ABF
:10A5100002D010BC1846704710BC002070470000E5
:10A5200070B50D4C05462078002812D000200B4E47
:10A530002070E9B23046FEF741FB02213046FEF7BB
:10A54000CDFA0028F9D002213046FEF7B5FA0120F5
:10A550002070284670BD00002440002000480040C4
:10A56000F0B50878324F334D334E801E83B00C4621
:10A57000062859D201007944097949188F440225E7
:10A580005434543A01203070A0786876A078C0071F
:10A5900005D02A492A48FEF767F8387AA874B28AA3
:10A5A000002A06D0FF20F5307080032125480DF4E5
:10A5B00085D5F169002937D0002000900190052051
:10A5C0006A461070684688472EE000246C7601F0D9
:10A5D000DBFCF169002927D0009406206A4601942B
:10A5E0001070684688471FE01722A11C1648FDF727
:10A5F0002FFE19E0B8780001C0194030807D002896
:10A6000012D11C22A11C1148FDF722FE0F48A18A7D
:10A610000182E18A4182218B8182618BC1820B4957
:10A62000608A0883207F6874002003B0F0BD0000BA
:10A63000504D0020944C0020B04C0020594D00207B
:10A64000A74C0020040F00008E4C0020744C00200A
:10A65000F0B518460D46014685B022230322744802
:10A660000DF46AD201210446417028780B286ED27D
:10A6700001007944097949188F4405CDCDCD6F6A21
:10A68000BB23CDCD6C0001202070607069488179BA
:10A6900021710179A170C17961714179E170017A0B
:10A6A000A171417AE171817A2172C16900294ED08C
:10A6B0000020009002206A46107068460194884786
:10A6C000A9E00720207001206070684620F4C6D7FA
:10A6D000019F009EFDF7AAFD801960820025FDF70D
:10A6E000A5FD8119601900908170FDF79FFDC119CA
:10A6F00000986D1CEDB20175082DF0D30825FDF70B
:10A7000095FDB919401861196D1CEDB28870102DB6
:10A71000F5D3102020774848817809010818403087
:10A72000807D012877D11C22A11C4448FDF790FDB3
:10A730004248A18A0182E18A4182218B8182618B18
:10A74000C1823E49608A08833D48217F417462E0AE
:10A75000052000E00A2020705DE004222270687865
:10A76000012804D0002802D0022833D053E0012071
:10A77000304D6070287C002810D002A820F46ED7DD
:10A78000FDF754FD2F49FDF7F7FC2F4808180299F3
:10A7900040182E49FDF7F0FC009101E0E8680090B8
:10A7A000E969002907D00020029003206A46107250
:10A7B00002A8039288471021A01CFDF762FD0098B3
:10A7C000A0700098000AE0700098010C2171000E42
:10A7D000607120E01748C169002905D00020009071
:10A7E000019068460270884720460C380DF4D6D197
:10A7F00014E00620164D2070E878012811D01021B1
:10A80000A01CFDF73EFDA9886182E988A182298903
:10A81000E1820020207620460DF4CAD1002005B048
:10A82000F0BD10220B49A01CFDF712FDEBE7000064
:10A83000140E0000B04C0020504D0020744C00203D
:10A84000944C0020A0BB0D00A08601003F420F00E9
:10A85000D44D00205F4D002000B5084883B0026C45
:10A86000002A08D000200090029005206B46187046
:10A87000684601919047002003B000BD504D002074
:10A8800010B584B0FF2B19D0144C226C002A08D0CC
:10A8900000200090029006206B46187068460191D7
:10A8A000904703200DF406D2032814D1A26F002A8A
:10A8B00011D003210A480DF401D40CE0094801230A
:10A8C000007F03220102084808310DF435D1072129
:10A8D00001700DF46DD1002004B010BD504D00206A
:10A8E000090E0000B04D0020050E0000FFB51A460D
:10A8F0000C461D0A83B02B464D494EA0FEF762FC64
:10A90000524EFF2DB5707DD02902342303225048CA
:10A9100008310DF411D10546B078002701018919DD
:10A9200040318872B078218800018019403001815F
:10A93000B078617A000180194030C172B0786289C4
:10A940000001811940318A81A289CA81E089088287
:10A95000207C012802D0002807D00BE0B17801202C
:10A96000090189194031887504E0B0780001801927
:10A970004030877520883080607A307221460A31F5
:10A980003448FDF771FE02F023F900281BD0607AED
:10A99000012804D1032211462F480DF41DD102F0E5
:10A9A0001FF905280FD201007944097949188F440D
:10A9B00006060602060001212820415505E0052172
:10A9C0002820415501E028204755032105980DF422
:10A9D00083D117203086B178090189194031488226
:10A9E0001E48C068002803D003211D480DF4C6D2BC
:10A9F0001C48028D002A03D003211B480DF45ED3AE
:10AA0000306C00E00EE0002808D002206946009774
:10AA1000087002950194316C6846884728460DF409
:10AA2000C7D001E001F028FA002007B0F0BD000017
:10AA300017EC000125732C207369643A25642C639C
:10AA40006F6E6964783A25640D0A0000504D00204D
:10AA5000020E0000594D0020150D0000604E002030
:10AA6000030F0000D44D0020020F000030B50C464B
:10AA70001D0A83B089782A4615A0FEF7A3FB28019A
:10AA80001D4DFF2140194030817201F0C9FA0028A4
:10AA900003D1022103200DF41FD12A6C002A08D013
:10AAA00000200090029003206946087068460194D7
:10AAB000904710211148FDF7E4FB11480068002879
:10AAC00002D009200CF4F2D6002003B030BD000003
:10AAD000424C4520446973636F6E6E6563746564B0
:10AAE0002C7265736F6E3A25782C636F6E6964788B
:10AAF0003A2564200D0A0000504D00206F4D0020C3
:10AB0000100C002000B5084883B0C169002907D0A7
:10AB100000200090019009206A461070684688471E
:10AB2000002003B000BD0000B04C0020FFB591B084
:10AB30000D4612230322454814990CF4FDD7002139
:10AB40000446017042480078002865D04048407CA7
:10AB5000002836D03C216846FDF793FB01F0D0FD7C
:10AB6000002844D004A90F913949461EF0B23A2278
:10AB70008969504341186846091DFDF769FB68461D
:10AB8000008B2988884206D10822A91C0F98FDF75E
:10AB900083FB00280BD0207800280ED008A8407C2A
:10ABA000607410226946601CFDF752FB1FE029A06B
:10ABB000FEF708FB01202070F0E73006000ED3D12D
:10ABC0002AE02A482988008B884225D10822A91C1E
:10ABD0002748FDF761FB002809D101202070254896
:10ABE0001022407C60742149601CFDF731FB207805
:10ABF000002811D01648C169002907D00020009014
:10AC0000019007206A4610706846884720460CF479
:10AC1000CFD7002015B0F0BD0D48C169002907D07D
:10AC200000200090019008206A461070684688470E
:10AC300002230322104814990CF47ED701210170DD
:10AC4000062141700CF4B4D7E0E70000180E0000B4
:10AC5000B04C0020656469762672616E645F6E6236
:10AC6000206D617463680D0A00000000744C0020C0
:10AC7000844C0020944C0020040E000070B50C465B
:10AC800009781B481B4D1E46002904D0012912D00B
:10AC900002292BD11AE01C2331460CF44DD706466D
:10ACA00020783070287B70802A7B1349301DFDF797
:10ACB000CFFA304607E00A2331460CF43DD721781D
:10ACC0000170698941800CF473D70FE00A23314683
:10ACD0000CF432D721780170298C4180698C8180F5
:10ACE000A98CC180E98C01810CF462D7002070BD71
:10ACF0000B0E0000D44D0020E14D002010B50C4695
:10AD00004A78097803A0FEF75DFA207800F0C4FDC8
:10AD1000002010BD74785F7068793A25642C207229
:10AD2000785F7068793A25640D0A000005480A8842
:10AD300042861A0A120110180988403081820020C8
:10AD400070470000504D002030B5180AC04300067F
:10AD500083B00D46000E21D0190A0902E120062316
:10AD60000322000108310CF4E7D6044601202070CC
:10AD700002206080FF204130A0800B48026C002A36
:10AD800008D00020009004206946087068460195AC
:10AD90000294904720460CF40BD701E001F06CF8C8
:10ADA000002003B030BD0000504D002000B5084821
:10ADB00083B0026C002A08D0002000900290082086
:10ADC0006B461870684601919047002003B000BDA3
:10ADD000504D002070B518460C46014602230A4823
:10ADE0000CF4AAD605460949A07808736288211D8B
:10ADF0000748FDF72DFA0020687020782870284653
:10AE00000CF4D6D6002070BD0D0E0000D44D0020ED
:10AE1000E14D00204A780B48002A05D02030012A55
:10AE200008D0022A09D00AE00279012A07D109785C
:10AE3000C17004E00978017501E0097841750020CE
:10AE400070470000504D002070B54878002806D0AB
:10AE5000FF25124C01280BD0022816D01BE0104809
:10AE60000179062917D10721017100F073FF12E063
:10AE7000207DFF280FD001F06BF80A482575016985
:10AE8000002908D00020884705E0607DFF2802D017
:10AE900001F040F86575002070BD0000704D002085
:10AEA000504D0020604E002010B5032B06D010221C
:10AEB0000548891DFDF7CCF9002010BD0348017A33
:10AEC000034801F0D3FCF7E76F4D0020504D002000
:10AED000594D0020F0B54B788DB00D46002B04D0B5
:10AEE0002A78E549E5A0FEF76DF9EB4E287834465F
:10AEF00000272034A1287AD012DCE8490C911B28C5
:10AF000076D006DC012819D003287CD017286DD113
:10AF10004FE128286ED091286DD0A02866D152E14B
:10AF20000146A239092961D20A007A44127992189D
:10AF30009744FE5CFDFD5CFDFCFDFD00687800288B
:10AF400054D1012001F0D2FF01F000FD342303228F
:10AF50000721D3480CF4F0D503210170D1490446F0
:10AF60008A7842700122C276FB224284CE4AC28491
:10AF7000CE4A82840A88028487768A888280CA8838
:10AF8000C2800A892281487A8009032805D18878FD
:10AF90000522104201D10120A076A07E0422104398
:10AFA000A076C3486080C878012825D020461021AB
:10AFB0000A30FDF766F9316C002907D001206A4696
:10AFC000009710706846019502948847012000F0B0
:10AFD00063FC20460CF4ECD5012303220721B5487D
:10AFE0000CF4AAD51A2101700CF4E2D535E11EE16A
:10AFF000CAE008E069E049E0204610220A300C99D6
:10B00000FDF726F9D7E70097019702970397049772
:10B01000059706970797089709970A970B9701F0E6
:10B02000D7FD002805D0684601F0BEFB0AA801F054
:10B030008BFB01F0CDFD00280CD0684680790028FC
:10B0400008D108A8807B002804D00121684600F0C0
:10B05000F9FF02E1934C6946A0880880E0884880A7
:10B06000208988808F71102202A80C99FDF7F0F8D2
:10B07000E078012804D00697079708970997E4E736
:10B08000102206A80C99FDF7E3F8DEE7E07B002824
:10B0900013D111230322072187480CF44DD505460F
:10B0A000282028707F48C078012808D01021681C0B
:10B0B000FDF7E7F828460CF47BD5E773CDE01022C6
:10B0C000681C0C99FDF7C4F8F4E7012001F00EFFAD
:10B0D000012103200CF400D67848012444841F2069
:10B0E000049070480178490601D57F210491817848
:10B0F0000522114204D0FF220499813211430491A8
:10B100000088C00504D5032104984902084304902F
:10B1100008216B480191029003210B2304AA009798
:10B120000394C9026748FDF7B7FA02E079E04AE004
:10B130008BE0002846D1644806218786FF200590D1
:10B14000624801910290082305AA00970394604980
:10B150006048FDF7A1FA00287FD100F0E5FD002846
:10B160007BD1022103200CF4B7D5B079012808D097
:10B1700000F0AAFE58484078C0076ED001F0D2F91E
:10B180006BE000F079FE68E001F022FDE77300F06B
:10B19000CBFD002861D1022103200CF49DD5B079AC
:10B1A0000128EED000F090FE4B484078C007E5D172
:10B1B00053E06878002850D0F179481EF071474874
:10B1C00001F024FB49E07179491E052906D8A7281A
:10B1D00002D13079002806D100F0BCFD2878A428DF
:10B1E00001D0A72839D17079042806D0062804D0C8
:10B1F000082808D00C2830D10CE039480168002913
:10B200002BD0B07904E034480169002925D0012011
:10B21000884722E03048016900291ED00320884772
:10B220001BE03771FF20F0702075607515E0207D00
:10B23000FF2802D06878002802D000F089FE0CE0D8
:10B2400025484078C00799D107E0607DFF2802D0EB
:10B250006878002804D000F05DFE00200DB0F0BD3D
:10B26000A07D0028F9D01C4840788007F5D5E17D05
:10B270001C4801F0C5F8F0E702EC000125732C2012
:10B280006F70203D2025782C2073746174757320B5
:10B290003D2025780D0A0000504D00205F4D002014
:10B2A000040D0000D44D00200502000048080000F5
:10B2B000A08C0000190D0000230D0000B00B002031
:10B2C0006AEB0001D20B0020680B0020C2EB0001EA
:10B2D000011800009C0B0020604E0020594D0020FA
:10B2E000004E0020884D002070B500250C462846F1
:10B2F000401C0628FCDB254E2246307E31461A32A1
:10B30000C96906282AD203007B441B79DB189F44B5
:10B3100024020910171E0622A01CFCF7BDFF0028FE
:10B320001BD01BE0237E092000F00AFF002814D167
:10B3300014E0237E212000F003FF00280DD10DE052
:10B34000237E162000F0FCFE002806D106E0237EB6
:10B35000192000F0F5FE002800D001250C48807D62
:10B36000002811D17169002901D020468847002D9D
:10B370000AD03169002901D00220884701F054F930
:10B38000217AA01C01F03CF8002070BD604E002026
:10B39000704D002010B50A78000A000210434A7868
:10B3A000FF231B02120298431A4010438A781B02A3
:10B3B000120498431A401043C9780002000A090693
:10B3C0000843FCF73CFF002010BD10B510460CF4FC
:10B3D00071D4002010BD0020401C0628FCDB00209A
:10B3E00070470000F8B51C4617460D4610460CF491
:10B3F00061D4002811D1472001F014FD0646042332
:10B400003A46032106480CF497D3210A0170298893
:10B41000B288891A41800CF4CBD30020F8BD00001B
:10B420000D470000F8B517460C46472001F0FAFC1E
:10B4300021780646122901D013291BD1B068054690
:10B440000C351229C288018916D006230F480CF446
:10B4500073D369884180617801710CF4A9D3B06815
:10B46000002803D00CF458D20020B06000213846E8
:10B470000CF432D40020F8BD042305480CF45CD34E
:10B480006988018061788170E7E700000947000062
:10B490000747000000B5084883B0026C002A08D0B6
:10B4A00000200090029009206B46187068460191B8
:10B4B0009047002003B000BD504D002030B5104D26
:10B4C00083B0088828861C0A200140190A88403069
:10B4D00042822A6C0025002A07D0009507206B467F
:10B4E000029518706846019190470648A10040589F
:10B4F000002801D04030C574002003B030BD0000EA
:10B50000504D0020580B0020FFB581B00020009066
:10B510000E4603980CF4CED3002802D001284CD05C
:10B520004DE0142001F07EFC07463188FEF76FFEE7
:10B5300005462448092D36D27C68002C1ED021797E
:10B54000A94203D02468002CF9D117E0002C15D0B3
:10B550006379039A9B1D04990CF4EED2054630885A
:10B56000288000202871607968806279A11D681D9B
:10B57000FCF76EFE28460CF41BD320E03D740498C3
:10B58000010A7974384601F045FC014601230E4852
:10B59000039A0CF4D1D205700CF40AD3012103985C
:10B5A0000CF49AD30BE00623039A04990CF4C4D24A
:10B5B0003188018080210171DDE702200090009830
:10B5C00005B0F0BD140C000002140000FFB585B0FA
:10B5D0000E4607980CF46ED3002802D0022009B062
:10B5E000F0BD472001F01EFC029000206946087063
:10B5F0000898070A308801F0EEFE002469460546E7
:10B600008C8000281ED102981622016A68460078B4
:10B6100003465043024610328A5A5204920F1FD1F9
:10B620000A5C401C085C1E4900021018884217D1B1
:10B6300002AA03A9184601F0E1FD02986946C05D1F
:10B6400088800224A31D1748079A08990CF474D225
:10B650000746308838803D717C80002D15D019E078
:10B660003946029801F0D6FB014604230E48079A9A
:10B670000CF462D207706946097841800CF498D2C4
:10B68000012107980CF428D307E0224601A9781D70
:10B69000FCF7DEFD38460CF48BD2002009B0F0BD7B
:10B6A00002290000140C000004470000FFB58BB015
:10B6B0000C46472001F0B6FB0025694605900D7445
:10B6C0000E9804A9070A208801F085FE060061D1C2
:10B6D00005981622016A6846007C504302461032E3
:10B6E0008A5A5204920F3AD10A5C401C085C3049D5
:10B6F00000021018884232D102950395208800F08C
:10B7000093F802A9002300911A4608A9FCF7DCFF70
:10B710006846008C012109030840C043C004C017DB
:10B720002146401CFEF728FD0606360E32D168463B
:10B730000997007C0190A57907AA694601F05EFD92
:10B740006846028806A80799FCF782FD06A90998B1
:10B750000A460D5468460188019801F08DFD39466E
:10B76000059801F057FBA1880D9A891D8BB20146FF
:10B7700010480CF4E1D10546A288A11D801DFCF7FC
:10B7800067FD2F706846007C6880A088A8802846E6
:10B790000CF40ED2042308480D9A0E990CF4CCD167
:10B7A0002188018086700CF403D200200FB0F0BD18
:10B7B000022900000A470000160C0000F0B589B00D
:10B7C0000446FCF787FF05460026154F1BE006A937
:10B7D0002046FCF74FFF002302AA01A906A8009605
:10B7E000FCF77EFF68460089B84203D169460979B3
:10B7F000022911D00B49884203D1684600790228FA
:10B8000007D0641CA4B2A888A04202D8E888A0424D
:10B81000DDD2002009B0F0BD204609B0F0BD000027
:10B820000229000003280000F0B589B00446FCF7A7
:10B8300051FF05460026104F14E006A92046FCF7EC
:10B8400019FF002302AA01A906A80096FCF748FFE9
:10B8500068460089B84203D1641CA0B209B0F0BDAB
:10B86000641EA4B2A888A04202D8E888A042E4D20C
:10B87000002009B0F0BD000003280000054CFF25A2
:10B88000F53501212046FDF79BF9284602F064FAC0
:10B89000F7E70000000C014010B5A0230949022879
:10B8A00009D0002203280AD0042808D00B704A705F
:10B8B00000F0A2F810BD0B7080204870F8E7E0207F
:10B8C0000870F4E711400020F8B52A4920204860AC
:10B8D00029480121C163294905228A610021C163E8
:10B8E00027490B20086100F087F82748254A0263A2
:10B8F00026494163264B8363264CC4632748264D63
:10B900000560274E4660274981602749C160274965
:10B91000016127494161274981612749016328481D
:10B9200026494160274FC760274F07610262274AB7
:10B9300042628362C46205634663254A8263254A84
:10B94000C2632648244A0260184A4260244A826040
:10B950000163244981632448244A41688918244AA0
:10B96000914206D2234982680A63C2684A63006929
:10B970008863F8BD00100140C02702404025024006
:10B98000402702400259F80040280240025B85002F
:10B99000025A8000025D8500025F805080280240CC
:10B9A00002000878020A0800026EAC500259FC003E
:10B9B0000200C8001270131402700314026E2800F3
:10B9C000C0280240025D0500125B0500025B840096
:10B9D000020A0600026E2C5002C3BF00002902407A
:10B9E0001200AC00125D0500104000206F2895FF8A
:10B9F000AF590F00C026024030B415481549037DE9
:10BA0000154AFF2B06D1407DFF2803D1134840780B
:10BA1000C0070CD01248134B04789C604078D86162
:10BA200011480861114B8B62106030BC7047104B9D
:10BA30000B6110484861104C8C61104D8D62C862DA
:10BA40000F48086313600F485060946030BC704723
:10BA5000704D00200028024040280240604E002027
:10BA60001140002000270240127E0200127E0300D7
:10BA7000027E020002C2A00012C70000027E030084
:10BA800012C7800002C2E00082B000F02DFFFDF777
:10BA900083FE18A0FDF796FB01212448FDF794F8DA
:10BAA00040212348FDF790F80120FEF7EBF93721FC
:10BAB00010A002F095F8FF20F530FCF717FE0020EB
:10BAC000FEF7E0F901F0C6F802200024020200901F
:10BAD000234618A10194184802F0E0F901200090D3
:10BAE0000023802215A10194154802F0D7F902F035
:10BAF0004BF9FEE70D0A204E53494E4720726177FD
:10BB00002064617461207472616E73666572207363
:10BB100065727665722831323862697420555549EC
:10BB200044292064656D6F200D0A0000000C01405F
:10BB300000080140424C45006DA100014C45440005
:10BB40007DB8000110B50124E4022046FCF7FCFE9C
:10BB5000002805D02046FCF7F1FE104902200870AD
:10BB6000012424032046FCF7EFFE00280FD02046D6
:10BB7000FCF7E4FE00F0B8FE09A0FDF723FBBFF3DD
:10BB80004F8F0F490D48C860BFF34F8FFEE70D4838
:10BB90004068002800D0804710BD000080000020D1
:10BBA0004E5253542D3E4E5649435F53797374653C
:10BBB0006D52657365740D0A000000000400FA05FB
:10BBC00000ED00E040400020EFF3088400F08CFE20
:10BBD00015A0FDF7F7FA214621A0FDF7F3FA24A0FE
:10BBE00062682168FDF7EEFA29A0E268A168FDF716
:10BBF000E9FA2FA062692169FDF7E4FA34A0E2694D
:10BC0000A169FDF7DFFA3A480068002800D08047B4
:10BC1000384939A0FDF7D6FABFF34F8F3949384874
:10BC2000C860BFF34F8FFEE72A2A2A2A2A2A2A2A27
:10BC30002A2A2A2A2A2A486172644661756C74206D
:10BC40004552524F523A52454720494E464F2A2AB2
:10BC50002A2A2A2A2A2A2A2A2A2A2A2A2E0D0A00A7
:10BC60006D7370203D203078253038782E0D0A0015
:10BC7000723020203D203078253038782C20097211
:10BC8000312020203D203078253038782E0D0A00D4
:10BC9000723220203D203078253038782C200972EF
:10BCA000332020203D203078253038782E0D0A00B2
:10BCB000723132203D203078253038782C20096CC4
:10BCC000722020203D203078253038782E0D0A0053
:10BCD000706320203D203078253038782C2009787A
:10BCE000707372203D203078253038782E0D0A0090
:10BCF0004040002054EB000125730D0A00000000B5
:10BD00000400FA0500ED00E0064A11780A2907D27E
:10BD10008900891848601078401C10700120704715
:10BD200000207047D04C002010B5084C084AE1793B
:10BD300013780020994207D2880080184068804715
:10BD4000E079401CE071012010BD0000504D002042
:10BD5000D04C0020F8B5324D052629792846807947
:10BD6000304C08290CD20A007A4412799218974470
:10BD700003080D1313191C2A052801D0FDF792FDA5
:10BD8000F8BD022808D0FDF73DFFF8BD607B002814
:10BD900002D1E079002802D0FDF7D2FFF8BDFDF70F
:10BDA0006DFFF8BD06202871F8BD0223032207218C
:10BDB0001D480BF4C1D6A5210170E9784170072117
:10BDC00029716E7128E002230322072117480BF422
:10BDD000B3D60746A7203870E978797006206871D5
:10BDE0000020287103200BF465D7032812D0A8790E
:10BDF000012804D0022802D003280BD104E0207DC2
:10BE0000002801D0032003E0A07E002802D00420F7
:10BE1000A87100E0AE7138460BF4CAD6F8BD000038
:10BE2000504D0020404E0020A20D0000A30D000048
:10BE300010B5002804D0014660220C48FCF708FA2F
:10BE40000B490C48CA781C2A04D9427B002A01D12C
:10BE50001C22CA70C1781F2901D91F21C170017B22
:10BE6000E22901D9E221017310BD0000004E00203B
:10BE7000204E0020404E0020114901220879072859
:10BE80000CD08879002809D0012801D0052806D1D6
:10BE90000C48827B002A03D002200CE08A71704794
:10BEA000027D002A01D0032005E0807E002801D019
:10BEB000042000E00520887110B5FDF7F3FC10BDEB
:10BEC000504D0020404E002070B5104C0525A07943
:10BED000062809D201007944097949188F440202E1
:10BEE00004040403A57170BDA57102230322072178
:10BEF00007480BF421D6A5210170E1784170072194
:10BF0000217165710BF454D670BD0000504D0020B6
:10BF1000A20D000010B50B4C607DFF2810D002234D
:10BF20000322072108480BF407D6A7210170617D81
:10BF30004170064A00215171FF2161750BF438D61A
:10BF400010BD0000704D0020A30D0000504D0020DA
:10BF500010B50A4C207DFF280ED0022303220721B2
:10BF600007480BF4E9D5A7210170217D4170054AEE
:10BF7000002151710BF41CD610BD0000704D002043
:10BF8000A30D0000504D002010B508480223807812
:10BF900003220102064808310BF4CED501210170BD
:10BFA000132141700BF404D610BD0000504D002049
:10BFB000040E000010B584B0002804D001462A22E7
:10BFC0000E48FCF745F90EA00FC86C460FC40B4B8A
:10BFD000002069461C180A5C247922430A54401C3C
:10BFE000C0B20628F6D310220A48FCF731F90A49F4
:10BFF0000A48FCF739FB04B010BD0000D44D002006
:10C00000501921901F04D5624FA489AB90D0CF2343
:10C01000000000005F4D0020D84D0020FC000020F3
:10C020000020074B01460A01D2184032927AFF2ABB
:10C0300001D0401CC0B2491CC9B20329F3D37047D8
:10C04000504D0020F8B507460B46282043430D46C7
:10C05000032207210E489B1C0BF46ED59121017021
:10C06000002406464570002D0ED92046282148435D
:10C07000C1190022CA7180192822801CFCF7E8F837
:10C08000641CE4B2AC42F0D330460BF491D5F8BD59
:10C09000910D0000F8B57D262025F600184B194CAF
:10C0A0001949032812D00A6A01273A430A620A6A28
:10C0B0009207FCD50A6AAA430A6201281AD002280C
:10C0C0001AD01E60FCF718FB2060F8BD0F480F2740
:10C0D00082683F023A438260086A04221043086281
:10C0E000086A0007FCD5086A284308623D20000161
:10C0F0001E60E9E7064800E006481860E2E7000035
:10C100008C00002090000020001002400010014030
:10C11000D103000057040000084A11780A290AD206
:10C12000C9004368891800688B6048601078401C1B
:10C13000107001207047002070470000FC4C002068
:10C14000FFB581B01C00064618D01078411CA142F2
:10C1500014D8032C12D3401EC5B25078971CB0429D
:10C1600006D12A4638460299FCF796F8002808D0EE
:10C170007A19601B801E0406240EE6D1002005B04B
:10C18000F0BD012005B0F0BDF0B504466F4E70481B
:10C1900083B06D4FB168C1626E490163F16A81621B
:10C1A000F16B4163B16B816331467C22403138468B
:10C1B000FCF74EF800257D60FD607D626648B86240
:10C1C0007D64BD64FD643D666448B8666448386259
:10C1D000644865490570032008706448F9140160DB
:10C1E0000904016089140160F06861490746401E36
:10C1F0000088604B884200D01F60366E701E008839
:10C20000884200D05E6001200003009069460195DD
:10C210000D710820487101278F716846FCF7A2FB59
:10C2200084215548FCF72DF82A215448FCF729F8B9
:10C2300060215348FCF725F852484F490561456194
:10C240008561C561056245628562C562FF264E480B
:10C25000CE70067546750020020152184032401C0F
:10C26000C0B296720328F7D32068086460684864F7
:10C2700046486189C187217A4548032901D8417719
:10C2800000E0457701212020FCF7BCFD414A4249EE
:10C29000042000F059FD4249404808600A464149DF
:10C2A000052000F051FD404A4049072000F04CFDB8
:10C2B00040493F4808600A463F49082000F044FDD5
:10C2C0003E4A3F49092000F03FFD3E4805633E4895
:10C2D000414907703D4805703D4805703D4808607C
:10C2E00001203E49C00208803D494F2008703D4969
:10C2F000082008703C480721067046708670C1709F
:10C30000057145718571C57111483849C161384958
:10C31000016238494162002001F0CEFA364903201B
:10C320000BF41ED5002103200BF4D6D4002000F01E
:10C33000DDFD01230322072130480BF4FDD30770F4
:10C340000BF436D403B0F0BDC0090020008000011A
:10C35000C0000020C9BB00010D470020D1D9000159
:10C3600045BB0001C6000020D800002000E100E02D
:10C37000FEE7000040400020504D0020D44D00203A
:10C38000004E0020504E0020704D0020904D0020A7
:10C39000B04D0020804000208080010021E8000195
:10C3A000C0400020C08001000041002000DB0100EF
:10C3B000814100204041002040DB0100C0460020B8
:10C3C000C06102000070004060000020C900002031
:10C3D000610000200090D0036C0000206800002065
:10C3E0006300002064000020080100208DCD0001C2
:10C3F000B5CE000155CE000100ED0001020D000098
:10C40000F8B5404D0646687D3F4C0F46FF281CD0CE
:10C410002046C268002A03D003213C480BF44ED6C4
:10C420003A23032207213A480BF486D3A421017052
:10C43000697D0446417037480022017800291ED0EA
:10C440000121A170A28002701BE06D200223032253
:10C45000072140010BF470D3A22101702E49C97845
:10C4600041700BF4A5D3EF7531462C48FCF7FCF86E
:10C470000120A8756078022108436070F8BDA270A1
:10C48000A2800120E07019214901E1802248218128
:10C49000038CE381438C2382838C6382C38CA382CD
:10C4A000FF23E2824133184D23836D786D070DD54C
:10C4B0000525E5706181A181018CE184418C218594
:10C4C000818C6185C08CA085E28523863820075544
:10C4D000204631463230FCF7C7F8E078810703D5B3
:10C4E0000220FFF7D9F906E0400701D5032000E05C
:10C4F0000120FFF7D1F90A490C20487120460BF4BE
:10C5000057D3F8BD704D0020604E0020030F00008F
:10C51000A10D0000D04D0020D44D0020884D0020FA
:10C52000504D0020F8B52C4E2C4D317D01276878F8
:10C53000FF2941D0C1073ED0B84368702849002088
:10C5400008703A230322072126480BF4F5D204464B
:10C55000A4202070307D60702878A07068788006F4
:10C56000800F20716888E080A8882081E888E081B9
:10C5700028892082E7700120FFF78EF9687840074C
:10C580000AD5E07802210843E07068886081A888B5
:10C59000A0810320FFF780F96878000703D5E078D1
:10C5A0000C210843E0701049082048710020B07544
:10C5B00020460BF4FDD2F8BD384368706D2002238D
:10C5C0000322072140010BF4B7D2A12101700749D2
:10C5D000C9784170EDE70000704D0020604E0020EA
:10C5E000D04D0020A10D0000504D0020D44D002062
:10C5F00010B50A4C607DFF280ED0022303220721CC
:10C6000007480BF499D2A5210170617D4170054A5C
:10C610000D2151710BF4CCD210BD0000704D0020E3
:10C62000A20D0000504D002070B50B4C207DFF285E
:10C6300011D00A4D687909280DD002230322072161
:10C6400007480BF479D2A5210170217D41700921A1
:10C6500069710BF4ADD270BD704D0020504D0020BB
:10C66000A20D000010B504464088A1880246491C6E
:10C6700019234A43DB019A420FDC06280DD3228896
:10C6800090420AD3E2887D23DB009A4205D84B0012
:10C69000C9184843D100884204DD10A0FCF792FD80
:10C6A000002010BD14480E23807803220102134895
:10C6B00008310BF441D20921017021884180618841
:10C6C0008180A188C180E188018100214181491ECA
:10C6D00081810BF46DD2012010BD0000726571756F
:10C6E00065737420706172616D6574657273206525
:10C6F00072726F720D0A0000504D00200E0E000085
:10C7000010B5084A084B906901888478994206D18F
:10C71000917CA14204D20024FCF726FB00E0002417
:10C72000204610BDB04C0020341200000B4610B55E
:10C7300004493A228969504341181846091DFBF7FC
:10C7400087FD10BDB04C002010B590B004463C21D0
:10C750006846FBF796FDFFF7D3FF401EC0B269465F
:10C76000FFF7E4FF08A8807CA0710CA920460331E4
:10C77000FBF77AFF10B010BD10B590B004463C2115
:10C780006846FBF77EFDFFF7BBFF401EC0B269465F
:10C79000FFF7CCFF08A8007CA0710AA9204602314F
:10C7A000FBF762FF10B010BD10B590B004463C21FD
:10C7B0006846FBF766FDFFF7A3FF401EC0B269465F
:10C7C000FFF7B4FF0AA920460231FBF74DFF08A886
:10C7D000007CA071204606A9102208300231FBF728
:10C7E00037FD0848C17820461830012904D01021AF
:10C7F000FBF747FD10B010BD10220349FBF728FDE1
:10C8000010B010BDD44D00205F4D002070B590B029
:10C810000D460646FFF774FF002D23D0854221D830
:10C8200018230322072110480BF486D10446172051
:10C830002070012060703146A01CFBF715FF3C21E1
:10C840006846FBF71EFD6D1EE8B26946FFF76EFFF6
:10C85000204606A9102208300231FBF7F9FC2046D9
:10C860000BF4A6D110B070BD140D0000F3B58FB05D
:10C870000C463C216846FBF704FDFFF741FF012C05
:10C880001AD0002816D0154D0AAE0236441EE0B26A
:10C890003A22A969504341186846091DFBF7D8FCA4
:10C8A000062231460F98FBF7F7FC00280DD0200632
:10C8B000000EEBD111B0F0BD0949421ECA7101460C
:10C8C0000F98FFF7A3FF11B0F0BD06A9102205488D
:10C8D0000231FBF7BDFC11B0F0BD0000B04C0020F0
:10C8E000504D00206F4D002030B5002189B0084622
:10C8F000FCF77AFA0120FCF79DFA01210920FCF7E8
:10C900008DFA6846FCF7C2F80224009404200590D2
:10C91000694601940B48FCF75DF80B4D2846FCF77F
:10C92000CDF8E12040020690082069468883800106
:10C93000088400204884CC8306A92846FCF7D6F852
:10C9400009B030BD000C01400048004070B52B4CD0
:10C9500082B020688003FCD5294D687FFFF79AFBE1
:10C96000606A50210840402802D126A0FCF72AFC2A
:10C97000606A012630436062606AB04360622B489F
:10C98000C08F0A2811D9E16932071143E1612849B2
:10C990004A6832434A602849264A0A6003224A60AC
:10C9A0008860264808602648086068461EF456D607
:10C9B000244900980860687FFF252D02032811D0C4
:10C9C00000F048F9206BA8432063206B3F21490207
:10C9D00008432063206B30432063012203211A485F
:10C9E0000BF46CD319480168A94301601849086821
:10C9F000FF2212049043086002B070BD0010024094
:10CA0000B04D002049574447525354206973207356
:10CA100065742C2072657365742066726F6D204991
:10CA20005744472121210D0A00000000904D0020AD
:10CA3000401002405555000000300040AAAA0000F6
:10CA4000CCCC000048400020010F000000E400E0D2
:10CA500008E400E0F0B5D7B054A81EF4FFD54C4967
:10CA60000024886AC96A54990122411A09010909F6
:10CA7000D206914204D95499081A00010009414292
:10CA8000444E40290CDC7088002809D0401E70807C
:10CA90001422032140480BF411D3002057B0F0BDFD
:10CAA0003E48FF21569029316846FBF7EAFB707C2F
:10CAB000B569002832D0FFF723FE69468870B17C43
:10CAC0006F4688420BD23A2148430246291D381D41
:10CAD000FBF7BEFB69468878401C887008E03A2165
:10CAE000401E4843024629463E31381DFBF7B0FB45
:10CAF000694688783A214843C0190A46363856991B
:10CB0000FBF7A6FB264869460880B069FCF72CF9BC
:10CB1000FF2227326946B069FCF754F9FF20F5304F
:10CB2000708020A0FCF74EFB4A944B944C944D949B
:10CB30004E944F9450945194529418485394418D6C
:10CB400040AA1185818D5185C08D90851A4C48AAC7
:10CB5000257C9573102219494CA8FBF779FB1848DE
:10CB6000C078012804D11022164950A8FBF770FBA9
:10CB700001261548002DC67306D1A07C002803D0DD
:10CB800001214AA8FFF75EFA1048067085E7000009
:10CB9000C0800240B04C0020040F0000744C002004
:10CBA00034120000426F6E6420696E666F207374E9
:10CBB0006F7265640D0A0000944C00208E4C0020BA
:10CBC000D44D00205F4D0020704D0020D04D00203E
:10CBD00002480078002800D001207047B04C0020A7
:10CBE0000148007970470000B04C002070B517492B
:10CBF0003CC80E4684B040363CC643680268806834
:10CC00004B65134C0A658865607C002818D00025A8
:10CC100069460D72FCF7BAF8FFF772FD69460872B3
:10CC2000E1690126002906D068460095067002A831
:10CC30000190684688476846007A002802D026702E
:10CC400004B070BD257004B070BD0000744C0020AD
:10CC5000B04C002004490868401C0860012801D03D
:10CC600001207047002070472840002003490868D1
:10CC7000002802D0401E0860012070472840002094
:10CC8000F8B50C462849294B4118294F294A002656
:10CC9000069D002908D0012922D0274940180A28DA
:10CCA0002FD301202870F8BD20780A2838D22149D6
:10CCB00080000958214A914203D11E490E501E504E
:10CCC0002EE0B9422CD10322082311461C480AF455
:10CCD00033D721780170616841600AF469D71FE099
:10CCE00020780A281CD280001158B94218D119584E
:10CCF0001150207813496268401803210BF4DED1EB
:10CD00000EE0C0B20A280BD284001159002907D0C6
:10CD1000B94205D0094FB94202D016511E51884779
:10CD20002E700020F8BD0000FBF0FFFF4C4C0020EF
:10CD3000CBDA0001244C0020F9F0FFFFC9DA000132
:10CD4000060F0000070F0000102819D230B40D4C58
:10CD500083001B199D6989032D0B2D03090D0D43BC
:10CD60009D619969084D920992052940920A1143E3
:10CD700099610122616982401143616130BC704751
:10CD80007047000000200240FF0FC0FFF3B50546CA
:10CD900081B00026408800F003F901000AD01C4F42
:10CDA0006A88002014234343DB195B8A934203D132
:10CDB00042262AE0402628E0401CC0B20A28F1D3CF
:10CDC000002E22D1002414206043C019408AFF287D
:10CDD00006D0641CE4B20A2CF5D30A2C14D014E05B
:10CDE00028460830009014206043C0190E686B7804
:10CDF000AA880746A91DB0470600EED16888788248
:10CE00000298398A0180E8E74B26304603B0F0BD2E
:10CE1000084B002002885004400CD20B01D00902BC
:10CE20000843704710B40024094A214614234B4399
:10CE30009B185B8A834204D1142041438818C4683C
:10CE400003E0491CC9B20A29F0D3204610BC704740
:10CE5000084B002030B4FF23040AC5B20A49002061
:10CE6000142242435218128AAA4204D11422504377
:10CE70004018438A03E0401CC0B20A28F0D32002C5
:10CE800030BC184370470000084B0020084A117856
:10CE90000A290AD2C9004368891800688B60486073
:10CEA0001078401C1070012070470020704700006F
:10CEB000D04B002030B4FF23040AC5B20A49002039
:10CEC000142242435218528AAA4204D114225043D7
:10CED0004018038A03E0401CC0B20A28F0D32002A5
:10CEE00030BC184370470000084B0020F1B582B0F9
:10CEF0000299294E0020002900D1307000250298A7
:10CF0000002804D0012834D002283ED10FE0294661
:10CF100014225143214A284609308C182082C0B27D
:10CF20000AF438D7207C21460AF41AD72DE0284687
:10CF300014214843194900234718B87C00903078E1
:10CF40001C4600280DD9E0008019828800998A4289
:10CF500002D1806880470346641C3078E4B2A04266
:10CF6000F1D8002B02D0596838468847387C0AF43B
:10CF700035D71422094B6A430021D018FF24C16021
:10CF8000448299504160018141816D1CEDB20A2DAE
:10CF9000B5D303B0F0BD0000D04B0020084B0020FB
:10CFA00070B50146094DCEB200202978044600290B
:10CFB0000BD9E10049198A88B24201D188688047BB
:10CFC000641C2978E4B2A142F3D870BDD04B002094
:10CFD000F8B5134E0F46756904463068001D00F021
:10CFE0002DFE601C07D1002F05D031680D48091DAA
:10CFF00000F05EFEF8BD30682C1944603168AC4228
:10D0000004D2B068091D00F03AFEF8BD7068091D31
:10D0100000F035FE306B8442F7D23463F8BD000077
:10D02000504700202C580020114D124E124FE86836
:10D03000002817D000F048FEF068C468201D00F0FA
:10D04000FDFD2869401E2861E868401EE86000F088
:10D0500047FE206B00F052FE204600F04FFEE868CD
:10D060000028E7D138680128E1D900F069FEDEE741
:10D0700050470020185800205057002030B4124963
:10D0800000E011460A688242FBD34B685C18844278
:10D0900003D1406818184860084643681C18944239
:10D0A0000CD10A4C2468A24206D052689A184260F9
:10D0B0000A681268026002E0046000E002608142D7
:10D0C00000D0086030BC70479C4700208C4700208F
:10D0D00003480068401C72B600D0FEE7FEE700007F
:10D0E000A4470020F8B50446002500F075FE374E31
:10D0F00000273068364A002801D0F0681BE005217F
:10D1000034480903430705D0C01DC008314BC00097
:10D11000C31AC91A41180839C908C90057601060F4
:10D1200031604F600B1A0F6043600160B3600120F3
:10D13000C0077360F06004423FD1002C3DD0204610
:10D140000830410708D04107490F0823591A081829
:10D15000410701D072B6FEE700282ED071688842E0
:10D160002BD81B49146801E02146144662688242AC
:10D1700002D22268002AF7D1326894421DD00D688D
:10D1800022680A60616808350A1A102A09D921182C
:10D190004B0701D072B6FEE74A6060600846FFF7B1
:10D1A0006DFF61687068401A7060B268904200D28A
:10D1B000B060F06827600143616000F095FF680788
:10D1C00001D072B6FEE72846F8BD00008C4700206B
:10D1D0009C4700204058002010B40124031F24065F
:10D1E0001C601B1F1960191F034B0B6014390A6068
:10D1F00010BC403870470000D1D0000170B5064621
:10D2000014460D464720FFF70DFE0369002B0DD095
:10D210001879B04207D158792880981D2060002BDA
:10D2200004D0002070BD1B68002BF1D100202880A5
:10D2300020600A2070BD000070B516460C461046EE
:10D240000AF438D5002813D14720FFF7EBFD054637
:10D2500006233246194607480AF46ED4A988628824
:10D2600089180180A1884180A17901710AF4A0D4B4
:10D27000002070BD180C0000F7B506460D4647208B
:10D28000FFF7D0FD04690746002C14D02079B04286
:10D290000BD16079A8420CD0384621461030FBF7FC
:10D2A00007FA20460AF438D305E02468002CEDD1B3
:10D2B00001E0002C0AD12846012108300AF4B6D337
:10D2C0000446014638461030FBF7F8F926716571BF
:10D2D0002A46A01D0299FAF7BBFF002003B0F0BD5B
:10D2E000F8B5C5680124287F0F4601281ADD0E4EC7
:10D2F0002046162250430246296A10328A5A5204A6
:10D30000920F0BD10A5C401C085C00021018B0425E
:10D3100004D1E1B20022384600F050F9287F641CA5
:10D32000A042E5DCF8BD000002290000F8B5C568A0
:10D330000124287F0F4601281ADD0E4E20461622B2
:10D3400050430246296A10328A5A5204920F0BD176
:10D350000A5C401C085C00021018B04204D1E1B223
:10D360000022384600F02AF9287F641CA042E5DC40
:10D37000F8BD00000229000070B5C46805462069A8
:10D38000002803D00020002802D00EE00120FAE798
:10D39000264610363046FBF779F90AF4BDD22069EB
:10D3A000002808D000210029F4D00020E8602046A1
:10D3B0000AF4B2D270BD0121F5E710B5044647204A
:10D3C000FFF730FD82790021A24202D9808800193E
:10D3D00081B2084610BD70B504460D464720FFF7E0
:10D3E00021FD014680888022A04206D88979411813
:10D3F000A14202D9201A28700022104670BDFFB544
:10D4000085B00E9D0646297801208840401E049074
:10D4100018460E210840328A69681F464030019242
:10D4200000230390009302912B7804AAA968069820
:10D43000FBF768F9009000282AD1012128200AF47E
:10D44000F5D20446AA686968286862622162E061D0
:10D45000F46006980188A180217FA171F80701D0AE
:10D460000120C003079908432080308A608047204C
:10D470007082304600F0BCF820461030FBF712F9FD
:10D48000217F206A00F008F8308A00210AF424D4B1
:10D49000009809B0F0BD0000F3B583B00020019002
:10D4A00004980125012845DD1621039A694388184F
:10D4B000028A5204920F39D1039A4078515C0002DB
:10D4C00009181D48814231D101A80290EFB204260B
:10D4D0004720FFF7A7FC00900469002C14D02079A6
:10D4E000B8420BD16079B0420CD000982146103080
:10D4F000FBF7DEF820460AF40FD205E02468002C82
:10D50000EDD101E0002C0AD13046012108300AF4A7
:10D510008DD20446014600981030FBF7CFF82771F2
:10D5200066713246A01D0299FAF792FE04986D1CAE
:10D530008542B9DB05B0F0BD022900000048704704
:10D5400098E7000170B5064613480D46007800289C
:10D550001BD04720FFF7AEFCA91D8BB2014603226A
:10D560000E480AF4E9D204460D482A468078207015
:10D570000120607005206080A5803146A01DFAF76B
:10D5800067FE20460AF414D370BD064900200870D7
:10D5900005A0FBF717FE70BD3747002006470000C7
:10D5A000504D0020394700204E6F7420656E616237
:10D5B0006C65206E6F746966790D0A0070B584B071
:10D5C0000E461446054601AA69463046FFF716FE88
:10D5D0006846028802A80199FAF73AFE02A8445563
:10D5E0000246684601883046FFF746FE04B070BD2B
:10D5F00010B504464720FFF715FC044921600921B6
:10D600006181183060600120208110BDA8E7000111
:10D61000FFB583B00C464720FFF704FC0546808821
:10D6200061882678401887B205980AF443D3012808
:10D6300007D03846FEF7C2F86946FFF7CCFE00284F
:10D6400002D0022007B0F0BD012105980AF444D3AE
:10D650000C3C0020AC60287368460078687301AA0F
:10D6600002A9FFF7CBFDA86801990446895D0C3437
:10D67000890720D5A188C28808318BB23102C12028
:10D680000001891D0AF458D2064613203070A8887C
:10D6900061884018B080A088F0803046A288A11D23
:10D6A0000830FAF7D5FD30460AF482D201210598F8
:10D6B0000AF412D301E00AF42FD1012007B0F0BD23
:10D6C00010B500F003FA002010BD0000FFB583B0D4
:10D6D0000C464720FFF7A6FB054680886188267820
:10D6E000401887B205980AF4E5D201280ED03846D2
:10D6F000FEF764F86946FFF76EFE002809D0014680
:10D700001FA0FBF75FFD022007B0F0BD022007B0AD
:10D71000F0BD0C3CAC602E7368460078687301AABB
:10D7200002A9FFF76BFDA86801990446895D0C34D6
:10D73000890720D0A188C28808318BB23102C1206C
:10D740000001891D0AF4F8D1064612203070A8881D
:10D7500061884018B080A088F0803046A288A11D62
:10D760000830FAF775FD30460AF422D201210598F7
:10D770000AF4B2D201E00AF4CFD0012007B0F0BD24
:10D78000737461747573206572723A25640D0A00B2
:10D7900010B50C464720FFF745FB80886188A31D24
:10D7A000401880B2A1880022FCF780FC002010BD48
:10D7B00010B508460022898801E0521C92B29142BD
:10D7C000FBD84288022A0DD0062A0ED102290CD19C
:10D7D0008179C07908180649012801D0002804D1B0
:10D7E000087002E0801DFCF7DBFB002010BD00008C
:10D7F00037470020F8B518460D46014605260BA709
:10D800000D230C480AF498D104460020A071287812
:10D810002070A6806888608032463946E01DFAF79D
:10D8200017FD20460AF4C4D10020F8BD4E53494EDE
:10D83000470000000547000070B516460C4610462C
:10D840000AF438D2012818D1A1791A48002916D033
:10D850002178062309023246891D0AF46DD1054656
:10D86000A078FFF7AAFD28808020287128460AF4B6
:10D870009FD1002130460AF42FD2002070BDA1882C
:10D880003246891D8BB221780902891D0AF454D1D0
:10D890000546A078FFF791FD288000202871A08818
:10D8A0006880A288E11D681DFAF7D2FC28460AF4B8
:10D8B0007FD1DEE7140C000010B5012400206407BE
:10D8C00020600AF48FD02E4802882E48016800207C
:10D8D0000AF414D12C4802882C48016801200AF46B
:10D8E0000DD12B48008882B22A48016802200AF430
:10D8F00005D12948008882B22848016803200AF42B
:10D90000FDD02748416AF0221143416225481DF4A9
:10D91000E7D02648244901602549416125498160B5
:10D920002549C160254981612549C16126492548AC
:10D930008863FDF7C9FF2068C0B2FAF7E9FE234803
:10D940000078002806D000201DF410D401460020E5
:10D9500002F4C6D22068C0B203F464D2FAF7DEFE45
:10D960002068C0B21DF48ED12068C0B21DF498D1D9
:10D970002068C0B21DF456D30120206010BD000005
:10D980001C0100201801002024010020200100209B
:10D9900034010020300100202C010020280100204B
:10D9A0004025024074020020500250008080024056
:10D9B00000080F0058086A00420500000F05050620
:10D9C0000F000F034000D0004080024062000020A2
:10D9D000F0B5314C83B0E06980075AD5022020624F
:10D9E000A56B08201DF466D401201DF471D42B49C9
:10D9F0000027086940194608B219801A08612848AA
:10DA00000068FAF737FD0022264BFAF7BBFC0191BC
:10DA100000903E212846FAF787FE80197941FAF7EF
:10DA200037FD019B009AFAF745FCFAF73FFD0546E2
:10DA30001D4A0023FAF7CAFB06461B49FAF774FE93
:10DA40001A49281A081A81B222041948324342603E
:10DA50000160206B0821884308432063A0690721E7
:10DA600009078843A061A169012081430143A161A5
:10DA70002062FDF729FF0F48104A00784100411845
:10DA80000D4808184178D1610D498078C8600D486B
:10DA9000077003B0F0BD000000800240A802002023
:10DAA0009000002000408F407102000070020000D2
:10DAB0004080024010400020B8E6000140250240AE
:10DAC000802502408000002070477047F0B52C4F41
:10DAD0007D20F968C000431AB868FFB0012282B007
:10DAE0009DB2814202D2401A84B204E0814232D90E
:10DAF000181884B2BA702348F988008EC01E884274
:10DB000000DDF880F888844200D904467A701C4A07
:10DB10001D48D268B9788618002921D0AC421FD997
:10DB2000012149026846FAF7ACFB2A4631466846AD
:10DB3000FAF78EFB661B6846401932461249FAF71F
:10DB400087FB21466846FFF7FDFC7D21C900304672
:10DB5000FAF728FB0EE0002078707FB002B0F0BD2D
:10DB600021463046FFF7EEFCF8687D210019C90018
:10DB7000FAF702FB0020F960B8707FB002B0F0BD88
:10DB800038470020504D0020804F002070B51148CC
:10DB9000FAF7A2FEFF210131081A0F4D84B2A888BE
:10DBA0000E4A84420CD2091A89B21018FCF7A2F965
:10DBB000002C03D021460948FCF79CF9AC8070BDCD
:10DBC0008442FCD9211A89B21018FCF793F9AC8071
:10DBD00070BD00001C00024038470020804E00202D
:10DBE00030B5134C8BB02278002A02D000200BB045
:10DBF00030BD01901020039102900E4A0020009247
:10DC0000802105910490032109030B4D0690079094
:10DC1000089009910A9069462846FAF767FE0121A3
:10DC200021702846FAF74CFE01200BB030BD0000F1
:10DC300038470020043801400800024043688268E9
:10DC400001699A60836842685A604A68824201D1D9
:10DC500082684A60002202610868401E0860086805
:10DC600070470146083100224160D243C1608260A2
:10DC7000016100210160704700210161704730B4EB
:10DC80000C68621C02D00246083202E0026904E01D
:10DC90001A4653681D68A542FAD953684B609960CB
:10DCA0008A60516008610168491C016030BC70479E
:10DCB00042684A6093688B6093685960916008611C
:10DCC0000168491C0160704772B604480168491C2C
:10DCD0000160BFF34F8FBFF36F8F7047A4470020E1
:10DCE00005490868002804D0401E086000D162B6CB
:10DCF000704772B6FEE70000A447002000281CD041
:10DD000070B504460D4D083C6068E968084201D1D1
:10DD100072B6FEE72268002A01D072B6FEE7884399
:10DD2000606000F059F860686968401868602046D3
:10DD3000FFF7A4F900F0D8F970BD70478C470020B8
:10DD40000120044900074860BFF34F8FBFF36F8F76
:10DD50007047000000ED00E010B500280FD0094921
:10DD60008A6B002A01D072B6FEE78A6B521C8A6366
:10DD70000021FFF72DF900F0B7F9002801D1FFF7D6
:10DD8000DFFF10BD5047002010B582B00D480024C1
:10DD90000190234680220CA100940D4800F07EF8EB
:10DDA000012803D0401C0BD172B6FEE772B60021E9
:10DDB0000848C94301630121C161446100F046F88C
:10DDC00002B010BD8447002049444C4500000000CB
:10DDD00029D00001504700200248816B491C816313
:10DDE0007047000050470020164B986B002802D067
:10DDF0000120586270470020586298691421024639
:10DE00004A4311498A58002A0AD1002806D0142210
:10DE1000401E42438A58002AF7D001E072B6FEE75E
:10DE2000142210B4424351184A680C465268083410
:10DE30004A60A24201D152684A60D1681960986173
:10DE400010BC7047504700205057002070B50F4855
:10DE5000016AFF22120411430162016A1202114396
:10DE600001620B4C00252561A5610A487D21C9008E
:10DE70000068FAF781F9401E6061072020610648BA
:10DE80000560FAF72FF9002070BD000000ED00E0FA
:10DE900000E000E000400020A4470020FFB585B06E
:10DEA00090000F9F0E9D0290FFF71CF906001ED0F8
:10DEB0005C20FFF717F9040016D02663059901913D
:10DEC0000899009130460299069EA5220391FAF71F
:10DED000D1F90399206B091F4018C008C0000290B7
:10DEE000400708D072B6FEE73046FFF707FF002074
:10DEF000C04309B0F0BD2118325C20310A75315C95
:10DF0000002902D0401C1028F5D3264600204036B8
:10DF1000F070072D00D30625E5620020E56420653A
:10DF2000201DFFF7A9FE20461830FFF7A5FE24614B
:10DF30000720411B6462A161002161653176009A6E
:10DF400001990298FFF748F92060002F00D03C604B
:10DF50002546FFF7B9FE284E3069401C3061306815
:10DF6000264F002803D0F069002821D026E0356034
:10DF70003069012822D1002414206043C019FFF722
:10DF800070FE641C072CF7D31D48FFF76AFE1D487E
:10DF9000FFF767FE1C48FFF764FE1C48FFF761FEB1
:10DFA0001B48FFF75EFE164870601430B06005E055
:10DFB0003068E96AC06A884200D83560F06A401C5F
:10DFC000F0626864E86AB169884200D9B0611421DE
:10DFD0004843C019291DFFF76BFEFFF781FEF0696A
:10DFE000002806D03068E96AC06A884201D2FFF78B
:10DFF000A7FE012009B0F0BD504700205057002077
:10E00000DC570020F057002004580020185800204A
:10E010002C580020F8B5324F0026B86B002808D0E5
:10E02000386A401C3862786A002800D001263046E1
:10E03000F8BD7D696D1C7D6115D178680068002888
:10E0400001D072B6FEE77868B9687960B860B86ADE
:10E05000401CB86278680068002813D07868C068EF
:10E06000C06840683863386B854211D378680068AF
:10E0700000280AD07868C068C4686068854211D2F8
:10E08000386305E00020C043ECE70020C04338635C
:10E0900038681421C06A4843124908580128C2D977
:10E0A0000126C0E7201DFFF7C9FDA06A002803D0A4
:10E0B00020461830FFF7C2FDE06AB969884200D9EE
:10E0C000B8611421484307494018211DFFF7F0FDAE
:10E0D000E06A3968C96A8842C8D30126C6E70000E9
:10E0E0005047002050570020F8B52E4D0027A86B50
:10E0F000002808D0FFF7E8FDA86B401EA863A86BB6
:10E10000002802D046E072B6FEE72869002841D018
:10E11000254E306800282AD0F068C46820461830A0
:10E12000FFF78CFD201DFFF789FDE06AA969884291
:10E1300000D9A861142148431C494018211DFFF74C
:10E14000B7FDE06A2968C96A884201D30120686284
:10E1500030680028E0D1002C09D0686829460068A2
:10E1600000281BD04868C068C068406808632C6AF3
:10E17000002C09D00126FFF74DFF002800D06E6269
:10E18000641EF8D100202862686A002802D00127A6
:10E19000FFF7D6FDFFF7A4FD3846F8BD0020C043C9
:10E1A000E4E70000504700200458002050570020AA
:10E1B00040BA7047C0BA70470138FDD170470000BF
:10E1C000F7B50325AD06286A82B016460C4640080E
:10E1D00040002862286A022108432862286A8007D2
:10E1E000FCD46620686001272F61A86AC005FCD5B1
:10E1F000992068602F61A86AC005FCD5FF20913086
:10E20000FFF7DAFFFF230133AB626846EF60352189
:10E2100069602F61A96AC905FCD5AB62A969EF6085
:10E22000C9B205226A602F61AA6AD205FCD5AB6229
:10E23000AA690902D2B211430180C80702D00320A3
:10E2400005B0F0BDAB626869FF21083188436861A1
:10E250006869C91E08436861029800024830686016
:10E260000820A860EE602F61A86AC005FCD5FF20D9
:10E270000130A8620023F61CB0080ED0B208114885
:10E28000006899006054060A09194E70060C000EC9
:10E290008E705B1CC8709A42F1D8FF200130A862D2
:10E2A0006869FF210831884368616869384368619B
:10E2B000286A800880002862286A38432862002083
:10E2C00005B0F0BD8000000C032080064169FF22EC
:10E2D000083291434161426901210A434261026A65
:10E2E000920892000262026A0A43026270470000CA
:10E2F000002003218906096A490849000322920681
:10E3000011621146096A0222114303229206116228
:10E3100000BF03218906096A022211400229F8D0B0
:10E32000D1010322920691620321D1609F215160A5
:10E330000121116100BF03218906896AFF22013290
:10E3400011409142F7D103229206916211468869E9
:10E350004969FF2208329143032292065161114616
:10E360004969012211430322920651611146096A4B
:10E370008908890011621146096A012211430322AA
:10E3800092061162704700000000010200000000C8
:10E39000010203040138FDD170470000F0B40324EA
:10E3A000A406236A5B085B002362236A02252B43D1
:10E3B0002362236A9B07FCD4FF230133A3626569B0
:10E3C000DE1DB543656165691E1D3543656100024B
:10E3D0006B3060600820A060E26001262661A06AC0
:10E3E000C005FCD5A3620023D21C90080ED095086E
:10E3F0000F4800689A008854070A52185770070C93
:10E40000000E97705B1CD0709D42F1D86069FF21AF
:10E41000083188436061606930436061206A800828
:10E4200080002062206A30432062F0BC00207047E8
:10E430008000000CF8B5064601200025C004864285
:10E4400001D90520F8BD0324A406206A4008400035
:10E450002062206A022108432062206A8007FCD4DF
:10E46000FF270137A76200F0BBF8002801D0032581
:10E4700015E00620606001212161A06AC005FCD57D
:10E48000A7623002203060602161A06AC005FCD51F
:10E49000A7620C4800F0C8F8002800D10225606986
:10E4A000FF21083188436061606901210843606190
:10E4B000206A800880002062206A08432062284683
:10E4C000F8BD0000E6960100F7B506460120C0043D
:10E4D00082B01546864202D9052005B0F0BD032062
:10E4E0008006016A490849000162016A022211435B
:10E4F0000162016A8907FCD4FF2101318162F2B215
:10E500008C1AA54200D8ACB20398009000F068F8CD
:10E51000002840D106214806416001210161816A3D
:10E52000C905FCD5FF2101310320800681624169C4
:10E53000FF22083291434161416904221143416144
:10E54000310232314160C4600022002C16D900989B
:10E5500087183B78F87819467B7800061B02194328
:10E56000BB781B04194301430802F978000A090625
:10E57000084319490860121DA242E8D30121032073
:10E5800080060161816AC905FCD5FF2101318162E4
:10E59000124800F049F8A54209D00398361900192D
:10E5A0002D1BFF2401340390A542ADD8ABE7032017
:10E5B00080064169FF22083291434161416901228D
:10E5C00011434161016A890889000162016A1143AE
:10E5D0000162002005B0F0BD8000000C1A060000AA
:10E5E00038B40125032080066A46C56035214160A4
:10E5F0000561816AC905FCD5FF2401348462816903
:10E60000C560CBB2052141600561816AC905FCD5B1
:10E61000846280691902C0B2014388B21180C007C8
:10E6200000D0012038BC7047F8B400210125032236
:10E6300092066B46D560352454601561946AE405F2
:10E64000FCD5FF27013797629469D560E4B20526AF
:10E6500056601561966AF605FCD5976296692402A4
:10E66000F6B234431C80E30722D0814202D9F8BCC1
:10E6700000207047032292066B46D5603524546013
:10E680001561491C946AE405FCD597629469D560CC
:10E69000E4B2052656601561966AF605FCD59762C8
:10E6A00092692402D2B21443A2B21C80D207DCD1F8
:10E6B000F8BC012070470000001713001710001766
:10E6C0000E0017090017040017000017180117148F
:10E6D00001171501171900000028000200000000B2
:10E6E0000328000200000000292A000200808000A8
:10E6F0000328000200000000242A0002008080009D
:10E700000328000200000000252A0002008080008B
:10E710000328000200000000272A00020080800079
:10E720000328000200000000262A0002008080006A
:10E730000328000200000000282A00020080800058
:10E740000328000200000000232A000200800800C5
:10E7500003280002000000002A2A000200800800AE
:10E760000328000200000000502A00020080070079
:10E7700045A20001D1A10001CFA10001CDA100015E
:10E7800000140000EDA20001130C000009B5000107
:10E7900003140000A9A30001FFD3000179D30001F5
:10E7A0002DD30001E1D20001130C0000CDB5000112
:10E7B000150C0000ADB60001170C0000E5B3000118
:10E7C000000C000025B4000106470000CDD6000172
:10E7D0000347000091D700010847000011D600014F
:10E7E0000E47000039D200010547000039D800016A
:10E7F000FFFF0000019C0001130E000051A6000164
:10E80000150E000061A50001170E00002DAB0001E0
:10E81000190E000005AB0001F0E700010500000043
:10E82000F7B586B0002002905C48154604695C4844
:10E830000E46824201D9054602E0002D00D1012595
:10E84000002C08D0A1880698814204D1E088B0420B
:10E8500001D1012002905348039084460698010498
:10E8600031430020002C1CD00A0CA7888BB29742A1
:10E8700007D1E7889F4204D1002807D021680160B2
:10E8800007E020462468002CEFD10AE061462268A8
:10E890000A602168002902D00020206001E0614662
:10E8A0004860002C07D10221102000F095F806994D
:10E8B00081800446C6802801052100F077F80746CC
:10E8C0007D200E464643EFF31085012080F310882B
:10E8D000684600F087F885F3108800980490C01906
:10E8E0000501019927202D098E1900010591864205
:10E8F00003D96D1C2D012D09361AE660A560039819
:10E90000294F86460020844670460068002813D0B0
:10E91000A268E1680091C36881680193531A1B01E2
:10E920001B09BB420AD2914203D1019A009991423C
:10E9300004D984460068E9E7724654602060604666
:10E94000002801D0046001E071460C601348029970
:10E950000069002901D1A04203D1C168806800F09C
:10E9600047F8EFF31084012080F3108802A800F02C
:10E9700039F884F31088039902980191291A090142
:10E9800009090090B94204D2A84205D101988642F3
:10E9900002D8032000F032F809B0F0BDC801002011
:10E9A000FFFF7F02D8010020FFFFFF0730B50B46B5
:10E9B000014600202022012409E00D46D5409D4259
:10E9C00005D31D469540491B2546954040191546DF
:10E9D000521E002DF1DC30BD03B40148019001BD91
:10E9E0002D7A010003B40148019001BD5DB602001B
:10E9F00003B40148019001BD9DB6020003B4014873
:10EA0000019001BDAD78010030B4C36882688868A8
:10EA1000084D141A2401C9682409AC4203D290425B
:10EA200004D18B4202D830BC0120704730BC00209A
:10EA300070470000FFFFFF070A0C838889B29342EA
:10EA400004D1C088884201D101207047002070475E
:10EA500070B4054600680022002810D00B0C868890
:10EA60008CB29E4207D1C688A64204D10168002A12
:10EA700007D0116006E0024600680028EFD170BCA4
:10EA8000704729600168002903D00021016070BC33
:10EA900070476A6070BC7047F0B5104F02688646D8
:10EAA0000025002A10D0C8688C6893688446E01A54
:10EAB00000010009D668B84208D2A34201D1B4458A
:10EAC00004D915461268ECE7704641600A60002DD3
:10EAD00001D02960F0BD70460160F0BDFFFFFF0767
:10EAE00070B584B004460E46EFF31085012080F324
:10EAF000108802A8FFF776FF85F310880298039923
:10EB0000024600900191A01A0001074900098842BD
:10EB100004D2A24205D10198864202D8012004B055
:10EB200070BD002004B070BDFFFFFF0730B583B09B
:10EB30000446EFF31085012080F310886846FFF744
:10EB400051FF85F31088019900986160206003B03F
:10EB500030BD00006E735F486172644661756C740D
:10EB60005F48616E646C657200000028000200005E
:10EB700000000328000200000000002A000A0080B4
:10EB800020000328000200000000012A000200808B
:10EB900002000328000200000000042A0002008096
:10EBA00008000328000200000000A62A00020080DE
:10EBB00001000328000200000000C92A00020080B2
:10EBC00001000028000200000000032800020000ED
:10EBD0000000052A0020008004000229000A00002D
:10EBE00002000328000200000000292B000A008018
:10EBF000100003280002000000002A2B0002008001
:10EC000010006761706D5F636D705F6576745F683B
:10EC1000616E646C657200676170635F636F6E6ED6
:10EC2000656374696F6E5F7265715F696E645F685A
:10EC3000616E646C65720000FFFF0000CD990001F9
:10EC4000A40D000015AE0001A50D000049AE0001A5
:10EC50001A0D000095B30001150D0000A9AE0001CA
:10EC6000000D0000D5AE00011C0D0000CBB300016B
:10EC7000A70D0000E9B20001A80D0000D7B3000104
:10EC8000020C0000BDB40001000C000095B40001AE
:10EC9000010E0000EDA800010F0E000049AD0001BB
:10ECA000110E0000ADAD00012C0E00002DAD0001D5
:10ECB000030E00006DAA00010A0E00007DAC0001E9
:10ECC000300E0000FDAC00010C0E0000D5AD0001BF
:10ECD000000E000059A80001090E000081A80001E3
:10ECE000010F0000ED9A0001020F0000959800014D
:10ECF000030F0000D19A0001040F000055CA000163
:10ED000038EC000136470020010019000214000011
:10ED100025A400010CED000101000000D0ED000170
:10ED20000300000001102EC78A0E7390E111C20883
:10ED30006027000000280000000000000000000024
:10ED40000000000000020000000003280000000096
:10ED500000000000000000000000000A00000000A9
:10ED600001002EC78A0E7390E111C20860270000CF
:10ED7000000400C0000201290000000000000000A3
:10ED8000000000000000000A0080140003280000BA
:10ED9000000000000000000000000000000A000069
:10EDA000000002002EC78A0E7390E111C20860278E
:10EDB0000000001000C00002022900000000000056
:10EDC0000000000000000000000A008014000000A5
:10EDD00004470000F5D700010A470000B1D7000141
:10EDE00007470000C1D6000108EE000100400020E6
:10EDF000AC0700001086000110F40001AC470020B1
:10EE000094680000F02A000011D490D00322A01AC8
:10EE1000FF01C1720113C202025020382B11D80D1C
:10EE2000490868496813F008FB0498EFF78EFF045F
:10EE300046C1888088FF22FFF79DFD2046FFF73AF4
:10EE4000FCB3E705B0F0BD981407D8011B20C80437
:10EE50002430D702100E4B1847FBFD064605203024
:10EE6000707580281699B181301D3946E5F773FD1C
:10EE70003046F9F70EFF0E222946422C45FD074089
:10EE800038112E0CD0534B052203212846FDF733B1
:10EE9000FE121E134B75162D05D0398F142902D082
:10EEA0001499897912E01010211176FAF74BF804C1
:10EEB0004D2859F9F7FBFE4C202851801112041BF4
:10EEC0002007771538B5049C103294014CA04738C0
:10EED000BD5143F84A26468F1839462036FD6D70DD
:10EEE0007D80311191C97FA0370E91224639781566
:10EEF000320F92F14A109203292BD0100C2873D0B4
:10EF0000F17D0F980CF00DF81014286FD068886907
:10EF1000460883F0B597B008780C460F901018207B
:10EF200014900F9848214843FE492246401806464F
:10EF300080361090F17F180991C56DA030169001B0
:10EF40004E180A274612922037F74A1552100F2AF8
:10EF5000D061783C2949D0432947D0787D100828D2
:10EF60007DD0F97D129814F0FCF9100E2878D06944
:10EF70008868468184687A297A1022040902084345
:10EF8000E97908430690A97A08A84172E97A817262
:10EF9000297BC17229460D310E380E91100AF02FCF
:10EFA000FAA878400733D5100E2132E0907E012870
:10EFB00006D0507E401E120610080E507603D00672
:10EFC000E03D21DB480106111012F0D2F9169A013A
:10EFD000211170A978D448C9075CD010089948233A
:10EFE00059430818101822A0300270FF20F0775201
:10EFF000E001220270A878CC49C0074CD09F984805
:10F000002358434020181442E0E97C08A8017329E2
:10F010007D4173697D8173A97DC108180D01742933
:10F020007E4174697E8174B189BC101E81F189C1F1
:10F0300081318A0182109940318A8F8283C98F0180
:10F0400084B188C183F18841841C21C18442101499
:10F0500072B848817808A8C17401E04DE11BE00254
:10F060002606752C2902D0CC100D02D4E87A800730
:10F0700005D5297B0E98380BF07EF908A908750391
:10F08000A90F0C1110402801D11698067060783C29
:10F090002870D030E1628869460A82A2884A82A23A
:10F0A000790A75E2794A75207A8875E07EC875A07C
:10F0B0008B0883E08B4883208C8883608CC88321F5
:10F0C00046243108A81018F0A4F9787A08A94871E4
:10F0D000B87A8871A08D69460885206B0B901E2038
:10F0E0000C90012018103E75387D0875B87D887524
:10F0F000A878C006C017401CC8758E486946028AA9
:10F100000A87428A4A87827D08A90A77C27D4A77A0
:10F11000027E8A77428B10A90A80828B4A80807F88
:10F12000087104A919A41332F91010984821484312
:10F130007C49401803907C301299101AF05DF90355
:10F1400098F97D8030817003990922A0310A7001FD
:10F1500021C170039817218166E18B49100F416628
:10F160000521C166016715996030C97E180E290412
:10F17000D072498161012102E02AE0241461817585
:10F180001F998182F97D12601009F6F8022802D2D7
:10F1900001214CF003F912281B05F906280CD20AAC
:10F1A000215F4A41438918FF318131497F89070333
:10F1B000D5FA7D7C2BFCF8961DFFF81699E0100C13
:10F1C00070FF20F077012014900920100AF0FBF85E
:10F1D00021460F3105911008284ED020233E222CC5
:10F1E00021564860100906460A20307014981428E9
:10F1F00001D01220100AE03C207070012030712CE8
:10F20000987080162D2CD0B01D5A1015F2F8F87D8C
:10F210007071E87A800706D52146304609310C30F6
:10F220002808F0E7F803E030460A1ADD20180A80C3
:10F230000705D53046123005303ADA1A1A121A107C
:10F2400015D0F8E08B3083208C7083608CB083B84D
:10F250007AB07730461010F0BFF83AE0287B707132
:10F2600029460D31B01D2CF0C2F8163EB4F83DE031
:10F27000149E1A2E9E3808A7F801210646019E1AF0
:10F280000D9E3C70703198280BF87D820709D5716E
:10F2900071B01D6A3CA5F80AB6180A30461DE0C0D8
:10F2A00007C00F701829B21A9978180BB081208CFA
:10F2B000F081608C3082782A74623C83F806601A90
:10F2C00016601777F8142101701008994180B97DF4
:10F2D00001713815F075F81598807E022826D160E6
:10F2E000781499084322D0082C1A0B2C1C61F812B0
:10F2F0002C100D61784170297881700FE040041462
:10F3000020C00624200A201A39041A400C111904BE
:10F3100014B1A2013304111F998180397E815613E3
:10F320004AF81E2017B0F0BD241DBA7047C0041063
:10F330000C03B40148019001BD919B02690C8BE163
:10F34000980C8B7D9F0C7C49FA010C8B09D30C8B9C
:10F350006D5B249B3D99488A900C8B5507308BD56B
:10F360009C188B397B1824796D011822210180416A
:10F3700080818070470A7802704B7843708A788267
:10F3800070CA78C2700B7903714A7942711A2C687D
:10F3900002600E033670472017497B41700570F1FB
:10F3A000F7F3FC2068F1F7A4FB256003B0F0BD2261
:10F3B000241220200A80024080C102400602101759
:10F3C000F8B54E784821F0B248432349214D411801
:10F3D0000C46AA7EA0346A27B014EDC3021710B5FC
:10F3E000074CE069100A0408D5FFF7F3FF0548123F
:10F3F00078180B2802D10120C00320621054295034
:10F400001AC6581AF4DB610265141AAA01410000F9
:00000001FF
